:03000000020257A2
:03000300D2C12245
:05000600D2C0D2C122AE
:03000B0002027579
:10000E00CD30E11520E00FC083C08288828C83CD75
:0C001E00F0D082D08322CDF222CDF62259
:10002A00CB30E11520E00FC083C08289828A83CB5E
:0C003A00F0D082D08322CBF322CBF7223F
:10004600ED30E11320E00EC083C08288828C83E00D
:10005600D082D08322E2226405700EC083C08288DB
:0B006600828C8393D082D08322E6229C
:10007100EB30E11320E00EC083C08289828A83E0E5
:10008100D082D08322E3226405700EC083C08289AE
:0B009100828A8393D082D08322E72272
:10009C0088F0A8817404C0E0C0F018E6C0E008E65F
:1000AC00C0E00886F018188001A3E0C608D5F0F966
:0200BC00F82228
:1000BE00EEC0E0EFC0E088F0E58124FDF8ECC6C0AC
:0900CE00E008EDC6C0E0A8F02234
:0C00D700E0A3FCE0A3FDE0A3FEE0FF229C
:0C00E300ECF0A3EDF0A3EEF0A3EFF02290
:1000EF0075F004AA83AB82D083D082E493A3CAC5F0
:1000FF0083CACBC582CBF0A3CAC583CACBC582CB7B
:08010F00D5F0E8C082C0832294
:10011700E5F06010C3EC13FCED13FDEE13FEEF13D7
:05012700FFD5F0F022FD
:10012C00120235C380021819E637F6DAF9020226F4
:10013C00E0A3FEE0FFEF8DF0A4CFC5F0CCA42CFC27
:09014C00EE60038DF0A42CFE22EC
:10015500C2D1C2D5EE30E707D2D1D2D5120202EC18
:1001650030E705B2D112020A12017D30D103120225
:100175000230D50312020A22BC000EBE0032EF8DFA
:10018500F08420D226FFADF0227B0075F008EF2F1A
:10019500FFEE33FEEB33FBEE9DEB9C4005FBEE9D46
:1001A500FE0FD5F0E9E4CECDCBCC227EFF7FFF223A
:1001B500EDB410005022EE8DF084FEEF54F045F0C2
:1001C500C48DF084C4FCEF540FC445F0C48DF08495
:1001D500FFADF0E4CC4FFF22EE8DF08420D2CC7E33
:1001E50008CEC5F0CDCBEF2FFFED33FD10D7079B24
:1001F5005005D5F0F1229BFD0FD5F0EA22C3E49F0F
:0D020500FFE49EFE22C3E49DFDE49CFC226C
:0C021200EE30E707E4C39FFFE49EFE22ED
:10021E0074F9800674FA800274FCD083D082258132
:07022E00F581C082C08322AC
:0F023500E5D054182407F8E58124FCF97A042257
:10024400EFB40A077F0D1202447F0A3099FDC29968
:030254008F99225D
:0F02570075813BE4787FF6D8FD75A0FF0215692D
:0702660075850175C01B2224
:03026D00C2C022EA
:05027000C2C0D2C22251
:10027500C0E0C083C082C0D0C002C003758C877542
:0B0285008AFF900033E0B46400504694
:10029000E004F0900005E0FAA3E0BA0004B4000125
:1002A000D3400CE014F0F49000057003E014F090DB
:0602B0000033E0B4325FF0
:1002B600900032E070057401F08005E4900032F0A1
:1002C600900031E004F0B40401D34043E4F0803FF1
:1002D600E4900033F0A3E004F0A3E0FAA3E0BA0050
:1002E60004B40001D3400CE014F0F4900035700320
:1002F600E014F0900039E0FAA3E0BA0004B400017B
:10030600D3400CE014F0F49000397003E014F09040
:090316000034E0B43B01D34010B7
:10031F00E4F0900038E004F09000377003E004F050
:0D032F00D003D002D0D0D082D083D0E032F5
:10033C002043686172676572205265736574202072
:10034C00002066726F6D205761746368646F67215B
:10035C00200020202057454C434F4D4520544F2022
:10036C0020200020534D41525420434841524745D0
:10037C0052202000436F707972696768742028439B
:10038C0029204279007777772E686F6262792D7217
:10039C00632E636F6D0020496E697469616C204D2A
:1003AC00656D6F7279200020506C65617365205704
:1003BC006169742E2E2E200020202A2A20455252AC
:1003CC004F52202A2A2020200020204D656D6F726C
:1003DC0079204661696C202020004C6F6164696E45
:1003EC00672042617474657279200046726F6D20CB
:1003FC004C6F636174696F6E2025326400204C6F02
:10040C006164696E672044656661756C740043684D
:10041C0061726765722066756E6374696F6E0069D0
:10042C00732064697361626C65642E202020200047
:10043C0044697363682E2066756E6374696F6E20F1
:10044C0000202020202025326443202534646D4177
:10045C00680020204E6F20426174746572792020F0
:10046C00202000202025352E3266562025352E32B0
:10047C006656730053544F502044495343484152DD
:10048C004745523F00204449534348415247452079
:10049C002020202020002020205761697420253343
:1004AC0064207365632E0020537461727420446958
:1004BC007363686172676500202020202020202053
:1004CC002020202020202020002020202020202040
:1004DC002020252B34646D41680025352E3266565C
:1004EC002025332E31664120253364730025352EAB
:1004FC003266562025332E316641202533646D003B
:10050C0025352E32665673202050574D20253264E7
:10051C00200053544F5020434841524745523F20EE
:10052C0020200020434841524745202020202020F5
:10053C002020202000205374617274204368617263
:10054C006765722020002046554C4C592043484189
:10055C0052474520202000204449534348415247EC
:10056C004520444F4E4520002055534552205445BC
:10057C00524D494E415445440020424154542E2082
:10058C004F5645522D564F4C540020424154542046
:10059C00444953434F4E4E45435400204C4F572033
:1005AC00535550504C5920564F4C540020444953ED
:1005BC0043482E2020252B34646D4168002044498B
:1005CC005343482E54494D45202533646D00204338
:1005DC0048415247452020252B34646D416800204A
:1005EC004348472E54494D452020202533646D0047
:1005FC002025352E326656702025352E32665665EE
:10060C00200020535550504C59202025352E326651
:10061C00567320002020204E6F202020202059656A
:05062C007320202000F6
:1006310090001BE0B401004007E0B40301D3400681
:10064100740190001BF0900020E0B40401D340033A
:100651007404F0900018E0FAA3E0FBBA0603B4407A
:10066100004009BA0704BB6C01D3400A900018741A
:1006710006F0A374A4F090000EE0FAA3E0FBBA0325
:1006810003B4E8004009BA0704BBD001D3400A9083
:10069100000E7405F0A37446F0900021E0FAA3E087
:1006A100FBBA0703B4D0004009BA0B04BBB801D3AD
:1006B100400A9000217408F0A374C4F0900015E082
:1006C100FAA3E0FBBA0103B4F4004009BA0404BB85
:1006D100B001D3400A9000157403F0A374E8F090C0
:1006E100001CE0B405004007E0B41901D3400674D2
:1006F1000F90001CF090001DE0B403004007E0B42F
:100701000A01D34006740590001DF090001EE0B46C
:100711001E00400AE0FB7A00B4F001D34006743CAD
:1007210090001EF0900012E0B41E00400AE0FB7A37
:1007310000B4F001D34006743C900012F090001315
:10074100E0FAA3E0FBBA0303B4E8004009BA0704E6
:10075100BBD001D3400A9000137405F0A37446F096
:010761002275
:100762004E6943444E694D484C69506F4C694F4E37
:04077200534C412083
:0D0776008B218A2289238D07E49000DDF09D
:0A0783009000DDE0B40216BF03137E
:10078D00AB21AA22A923744912002A0523E523705F
:10079D00020522EF25E025E0FE9000DDE02E90071A
:1007AD006293AD21AC22A82312000E0523E5237020
:0D07BD000205229000DDE004F0B404BA2231
:1007CA00900023E4F0A3F0A3F0A3F0A3F0A3F0A316
:1007DA00F0A3F0A3F0A3F0A3F0A3F0A3F0A3F022F8
:0A07EA0075D90275E90075F90022C7
:0607F4007F0112789B2238
:10080000A881058118EBC6C908CAC6CA08F67BFFCD
:10081000112ED0E0D0E0D0E0C082C08322D083D0BF
:1008200082EDC0E0ECC0E0E8C0E0C082C083E581BA
:10083000F82425F58108E8C9CBF709EAF709EBF7B1
:1008400009770009E924F6FA75F000C2D5E924FC1D
:10085000F8E924F9F9ECC0E0E8C0E0D1E51200467F
:10086000FFE92409F9D0E0F8D0E0FCEF605020D592
:1008700074B4250AE4FB74FFFCF7D2D580D3D1FE13
:1008800080CFFF20F71CBCFF067014D2F380C2ECAF
:10089000C0F075F00AA42FD0F030F703F78001FC08
:1008A00080AFB7FF03EF80F4E780E57F00D1FE194A
:1008B0001709800DEF24D0B40A0040C68093B6FF1C
:1008C000EAE581C39421F581E4FED0E0FFD082D037
:1008D00083D0E004600ED083D0821581158115810C
:1008E000C082C08322900F78E49360256FA36006D6
:1008F000A350F5A380F293FF400442F080BEE4A32E
:10090000938F83F582E4C2D130F705B7FF027700F9
:100910007340A1D3A380D1EAC8FDE620F703FC8091
:1009200001F71A1AEDF88094D2D17F7880027F58AF
:10093000D17990100421CCBCFF05B7FF02805AC0CA
:10094000F08AF0EAC92420F583E8FEECC0E0D1E5A6
:10095000120046FF601AC583C9C583F70B19E9C5A4
:1009600083F908B800010CEE2404F9E7C39B70E09A
:10097000D0E0FCE5F024FDFAD0F08B82A98309EEEB
:10098000C394FBF583F805828004E7F60809D58255
:10099000F9A9831819C2F0414F8AF0EAC9F583E832
:1009A000FED1E5120046FF6013EEC8CE8D82D1FE67
:1009B000AD82EEC8CE08B800EA0C80E7A983E5F066
:1009C00024FDFA01487F30D179900806C2F7D18919
:1009D000E8CAC9C88049D2F7EA147D0230F4047D20
:1009E0000424FEF8E68A83A88330E70DD2D1C3E45D
:1009F00096F618DDFAA8838000C2F7D179900A052F
:100A0000D189C9C8CAC9B1FF8015D179E618188043
:100A100004D1797425C2F7F70BCAC9C8CAC2F0E776
:100A2000FDE924002BF8B6300318DBFABB00080BF5
:100A300008BD00031B8013BDFF02800EEDC39BFEAB
:100A40004008600674305192EDFBEB70020148ECF7
:100A5000046023D39B401F601DFE7D2020F13830B1
:100A6000F3027D3030F023BD3018518E18EF30E6A0
:100A700001187111804030F03F71110B30F6390BC5
:100A80008036EF71111E30F6011E518E8028EE6007
:100A900005ED08F6DEFC2230F00771110B30F6018F
:100AA0000BE9FF2420F9E6F71918DBFAEDF719DE58
:100AB000FCEFF92420F8CCCBEB700201481919E8BF
:100AC000C0E0E6FFD1E50909EFD16AD0E0F818DB14
:100AD000EE090901481A1AD181900F6CE6086002EC
:100AE0002406936023F7190B30E504E4A380F3EBAD
:100AF000C0E0743AF7E924FCF908901004D1891891
:100B0000D0E02405FBE92404C8CAC9E92420F88000
:100B1000AC08EFF68FF030F604743008F622619BD3
:100B2000C2F79159BFFF0261ADEF60F22481FF204F
:100B3000E73618040FD113EBC39F60124010FDFE7F
:100B40000BE89FF8742EC618C6DDFC18805DF4040F
:100B5000FD7E000DE824F9F880057430F6180BDDF1
:100B6000F9742EF60B188043F4FD7E070DBD0700C7
:100B70004016E9FD097430F709E9C39870F7EDF9FB
:100B800080087430F60E0B08DDF8742EF6080B0B97
:100B90007430F6D113E8C39BF88010E92420F87470
:100BA00030F618742EF6187B027E00B1AD414AC2B1
:100BB000F78002D2F79159BFFF0280F1BF000E7497
:100BC00030F618742EF6087E007B02800EEF24812A
:100BD000FF18742EC608C6EBFE1E0BD113E8C39B8C
:100BE000F8EFC0E0B1ADD113D0E0FFC0F0E8C39B97
:0E0BF000F8E730F704746580027445F618EFDC
:100BFE0020E704762B8004762DF4041875F00A8411
:100C0E002430F618E5F02430F6EB2404FBD0F0D1B6
:100C1E002918B1FF61ADC2F78002D2F7D2F2915915
:100C2E00BFFF0261ADE7B4FF037406F7BF7B004060
:100C3E0016EF248120E706C397600C500A74822FAA
:100C4E00C7C397F7020B2917020BBCD179ECC0E092
:100C5E00C0F018E63308E63392D5186033B4FF407F
:100C6E00E6C2E76009900FBCC2D17B078007900FE8
:100C7E00C3D2D17B06E493F709A3DBF97B0330D112
:100C8E000A742B30D502742DF70B09197C80A184C0
:100C9E00EAC0E074307A08F709DAFC097C81A17D9C
:100CAE00CAC0E0EA75F010A4CAABF075F04DA42BE3
:100CBE00FBE435F0FCEA2410FAEB34C5FBEC34D936
:100CCE00FCE6C2E7FF75F056A4F42411C5F0F43427
:100CDE00C58FF0A42AE5F03BE43CFBC0E0E9C0E0A0
:100CEE00E8C0E0EBC0E020E707800812112C801F5F
:100CFE00F404FB121411D0F0D0E0F8C0E0187583A4
:100D0E000418E6C0E008D583F930F7DF121288D058
:100D1E00E0F8D0E02408F9EED2E7CE33EF332482A8
:100D2E00FAECFBD0E0FCE4C3CB33CBCD33CDCE33EA
:100D3E00CE33DAF37A0875F00A8460062430F71998
:100D4E001A0CE5F02430F7198BF0740AA4FBAFF0FF
:100D5E008DF0740AA42FFDAFF050010F8EF0740ABF
:100D6E00A42FFE743035F0F719DADDE9240AF9D034
:100D7E00E0FAE9D39AFBECFF247FFFCAC9C824FD31
:100D8E00FAE9FD09EF046003120F2FEDF909EF04E4
:100D9E006003120F2FEDF9D0F0D0E0FC7B0722E7B5
:100DAE00B4FF027406700820F0010E8E838016C305
:100DBE009E400EF583603674300BF618D583FA809C
:100DCE002CF404F583C0E0E9C0E0E8C0E0F92B04A0
:100DDE00F8EEC0E0EFC0E009120F2DD583FAD0E097
:100DEE00FFD0E0FED0E0F8D0E0F9D0E0FD08D12948
:100DFE0018D2F07F2D20D10C7F2B20F5077F2020DD
:100E0E00F602C2F0228982E92420F98B83E6F719D3
:100E1E0018D583F9A982E92420F822E9F582240164
:100E2E00F98B8330F22A20F027C2F2E608B42E02A4
:100E3E00D2F2D583F6E8C39BF88B8330F210E6B47A
:100E4E003005081BD583F7B42E07081B8006D2F297
:100E5E00E6F70908D583F9E9F8A98222BDFF051244
:100E6E000244800312000E09071922E9CAC8E924B8
:100E7E0001F922E9CAC8E92420F922A2F492D5C0C8
:100E8E00F0E582FD30D50623F582FD181818E685AB
:100E9E0083F084F620D5047B0180027B0308E5F005
:100EAE00D6C6C48583F084C4C6C445F0C48583F019
:100EBE0084D6DBE9E5F024F6500730D10224202455
:100ECE0007243AF70920D509DDC3D0F01818AB82F4
:100EDE0022DDB8181880F3E7F819E7FC19E7FDBD15
:100EEE00FF0122090907B70004190719221919224F
:100EFE00CACDE8C0E0E9C0E0E6FB08E6FA08E6F98C
:100F0E00EFBBFF05120244800A06B600031806085E
:100F1E0012002A080618D0E0F9D0E0F8CDCA22E96E
:100F2E00FD1BE7B4350FEBFE600709E719F709DE85
:100F3E00F718EDF92240EF09C3E899601AE719B4E2
:100F4E002E04F70980F104B43A067430F70980E7ED
:100F5E00F709E899FE80D1197431F70B80D4286E09
:100F6E00756C6C290049584450434C046C10620057
:100F7E00680023012D022B2020402E80002A091705
:100F8E006F09C578092858092E7309377509F96450
:100F9E0009D66909D6630A0A250A11700AD5660BA5
:100FAE0020650BB3450BAF670C28470C240020209F
:0B0FBE0020204E614E202020464E49AE
:100FC9001200D7EFB2E7FF80031200D7E58124FDB5
:100FD900F8F9E63308E63370060213B60213A504DE
:100FE90060FAEE33EF33700EE6FF18E6FE18E6FD01
:100FF90018E6FC0213B60460E3E58124FBF8D3ECA0
:101009009608ED9608EE9608EFC2E786F0C2F795C6
:10101900F0400FEFC6FF18EEC6FE18EDC6FD18EC3E
:10102900C6FC1213C7C3EB9FF5F0700EE58124FBD4
:10103900F9E4C3CC20D5730211049418605C400E06
:10104900E4FF19E7FE19E7FD19E7FC0210E0E4FFE8
:1010590030F405CEFCE4CDFF30F305E4CECDCCCFA2
:1010690030F21AE5D054184404F8EF54F0D6C4FF0E
:1010790008ECD6C4FC08EDD6C4FDEEC4FE740355D5
:10108900F06012F5F0C3EE13FEED13FDEC13FCEF67
:1010990013FFD5F0F030D55D8009E4CEFFE4FDFC07
:1010A90030D552C3E49FCC191919C797CD09C797F1
:1010B900CE09C797FF4E4D4C70140213B6DB0302DD
:1010C90013A9EC2CFCED33FDEE33FEEF33FFEF30CB
:1010D900E7EBECCFCECDFCEF30E70D0CBC00090DF2
:1010E900BD00050EBE00010BEB7005A2D102139DD8
:1010F900A2D10213B0E42FCC19191937CD0937CE73
:101109000937FF50090BEB700CA2D102139DEFCEEA
:10111900CDCCFF80C2EF13CE13CD13CC13FF80B714
:101129001200D7EF4E601AE58124FEF924FEF8E794
:1011390019477019EE33EF33B4FF030213A50213F5
:10114900A9E58124FDF8E63308E63380EB1213C7DD
:10115900248150082B5008A2D502139D2B50DFF78C
:10116900FAE61846197020B7800DEE33CAA2D513D6
:10117900FFCA13FE0213B6EC4D703CBE8046E6FC76
:1011890008E6FD08E680E4EC4D7039BE800280EE89
:10119900E4CEC7CDC6F5F008E4C6CCF9FBFFFA806A
:1011A90076E4CEC9E4CDCAE4FFCCFB803CE4C9CDEA
:1011B900CFCBECCACC8060E4F9FAFBFFCECDCCC52D
:1011C900F00880538CF0E660D8A4C5F0CDFAC5F0DC
:1011D900E6A42DCEF9C5F03400FDE6A42DC5F03402
:1011E90000FDCCFBC5F0CC7F0008E660C0A42EC58D
:1011F900F03C50010DCAFCC5F0CEE6A42AC5F03D6D
:1012090050010FC9FDC5F0CAE6A429C5F03F79010F
:10121900400119CBC5F0CF08E6A42AC5F03F500517
:101229000BBB000109CCC5F0FAE6A42CC5F03B5074
:101239000109CDC5F0CCE6A42DFDC5F039FE330872
:10124900500906B60011A2D502139DEA33FAEC3310
:10125900FCED33FDEE33FEEA30E7140CBC00100D53
:10126900BD000C0EBE000806B60004A2D580D9E662
:05127900A2D50213B034
:10127E00D083D0820213A91200D7EFC2E74E7003BB
:10128E000213A5C082C083E58124FBF8F9E6084667
:10129E0060DE1213C70FBF0006D083D08280E1EF4D
:1012AE0024805007C3CB9B500D80C5CB9B4007D0ED
:1012BE0083D08202139DF6F583EC4D701FBE801C09
:1012CE00E58124FBF8E583A2D513FFE692E7FE182D
:1012DE00E6FD18E6FCD083D0820213B6E58124FB2E
:1012EE00F8E6CEF618E6CDF618E6CCF6EFCCFFE82B
:1012FE002402F9F8E7FA19E7FB19E7FCE4F5F075B3
:10130E00821A758380801DE58303F58330E706A777
:10131E00F009E4F5F0C3EF33FFED33FDEE33FE409D
:10132E000C30E717C3EF9CED9BEE9A400EC3EF9C7B
:10133E00FFED9BFDEE9AFEE58342F0D582C9E7FAFA
:10134E0019E9F81919E720E7191ABA000302127EF3
:10135E00E5F025F0FFE633FC18E633FD18E633FE24
:10136E008009FE09E7FDE6FCE5F0FFEF30E7160C1D
:10137E00BC00120DBD000E0EBE000A0A7007D0830F
:0F138E00D08202139DEAA2D5D083D0820213B081
:10139D0074FF13FF7E80800774FF8001E4FFFEFD64
:1013AD00FC800613FFEE92E7FED0E0F8D0F0E58169
:1013BD0024FCF581C0F0E8C0E022E7D2E7C733098D
:1013CD00E733FB92D592D1EED2E7CE33EF33FF5018
:0413DD0002B2D52261
:1013E1003F8000003DCCCCCD3C23D70A3A83126F1D
:1013F10038D1B7173727C5AC358637BD33D6BF953A
:10140100322BCC7724E69595179ABE150A4FB11F5A
:10141100EB60105407700AEB543803241C12143C7F
:1014210022232312143CEB543870012203241CFBA9
:101431001200BEEB12143C12112C229013E1FC930A
:0E144100FF0CEC93FE0CEC93FD0CEC93FC22E4
:10144F001214958000EC3392D550031214837A2036
:10145F00C3EC20E712EF33FFEE33FEED33FDEC3339
:10146F00FC20E703DAEF22EA247DA2D513FFEC92EA
:10147F00E7CEFC22E4C39FFFE49EFEE49DFDE49CC7
:10148F00FC22C2D580C8EED2E7CE33EF3392D524FB
:10149F0081400CE4C2D5A2D513FC33FDFEFF2224FC
:1014AF00E0500474FF80EFF404FAE4CCCDCECF808B
:1014BF000DC3EF13FFEE13FEED13FDEC13FCDAF18A
:1014CF0020D507EECDFEEFCCFF22E4C39CFCE49DBC
:1014DF00FDE49EFEE49FCCFFEECDFE22EFC2E7FFC0
:1014EF0080A47A083392D5E4FDFEFF30D5031214A1
:1014FF0084EC334010EF33FFEE33FEED33FDEC336E
:10150F00FCDAEE80BEEA247EA2D513CC92E7CDCED4
:03151F00FF80B09A
:10152200E58124FEF88FF063F080E6F96480B5F07F
:101532001B188EF0E6B5F014188DF0E6B5F00D1814
:101542008CF0E6B5F006E4FFFE0213B68FF030F73A
:101552000689F030F701B340077F017E000213B61F
:0715620074FFFFFE0213B647
:101569007580FF7590FF75A0FF75B0FFE4FE7FFAE7
:101579001279D51278331207F4E4FF1279237589A9
:1015890001758C87758AFFD28C75A8821207EA12B9
:0815990077E6127A4C30C234EF
:1015A1001202707F017B057A03793C12794E7F022A
:1015B1007B057A03794D12794EC2B43080143081A3
:0115C1001118
:1015C20020B40312799E7E017FF41279D5B2B480E1
:1015D200E9D2B4308007208104D2008002C2007FA9
:1015E200017B057A03795E12794E7F027B057A03CD
:1015F200796F12794E7E077FD01279D57F017B05F4
:101602007A03798012794E7F027B057A03799112EF
:10161200794E7E037FE81279D57401900011F09023
:10162200001BF090001FF07404A3F09000187406E1
:10163200F0A374A4F090000E7405F0A37446F09029
:1016420000217408F0A374C4F09000157403F0A391
:1016520074E8F0740F90001CF07405A3F0743CA3BE
:10166200F0900012F0A37405F0A37446F0E4FFFEBC
:10167200900017F0127A83BE01028003021749BF5D
:07168200000280030217497A
:10168900740190001AF0E4FE7F01127A83EF900052
:1016990011F0E4FE7F02127A83EF90001BF0E4FE62
:1016A9007F03127A83EF90001FF0E4FE7F04127A21
:1016B90083EF900020F0E4FE7F05127A83EE90001C
:1016C90018F0A3EFF0E4FE7F06127A83EE90000E85
:1016D900F0A3EFF0E4FE7F07127A83EE900021F089
:1016E900A3EFF0E4FE7F08127A83EE900015F0A3D1
:1016F900EFF0E4FE7F09127A83EF90001CF0E4FE1C
:101709007F0A127A83EF90001DF0E4FE7F0B127AB4
:1017190083EF90001EF0E4FE7F0C127A83EF9000B5
:1017290012F0E4FE7F0D127A83EE900013F0A3EF1E
:10173900F0E4FE7F0E127A83EF900017F002189EF4
:101749007F017B057A0379A212794E7F027B057AA4
:101759000379B312794E127AF3E4FE7F0A1279D52E
:10176900E4FEFF127B46E4FDFEFF7C01127A55126E
:101779007B69E4FEFF127A83BE0102800302186FBF
:08178900BF0002800302186F8B
:10179100740190001AF0127AF3E4FE7F0A1279D5EF
:1017A100E4FE7F01900011E0FD7C00127A55E4FE19
:1017B1007F0290001BE0FD7C00127A55E4FE7F035E
:1017C10090001FE0FD7C00127A55E4FE7F0490003A
:1017D10020E0FD7C00127A55E4FE7F05900018E0C0
:1017E100FCA3E0FD127A55E4FE7F0690000EE0FCBA
:1017F100A3E0FD127A55E4FE7F07900021E0FCA3EF
:10180100E0FD127A55E4FE7F08900015E0FCA3E0AC
:10181100FD127A55E4FE7F0990001CE0FD7C001268
:101821007A55E4FE7F0A90001DE0FD7C00127A5596
:10183100E4FE7F0B90001EE0FD7C00127A55E4FE71
:101841007F0C900012E0FD7C00127A55E4FE7F0DC2
:10185100900013E0FCA3E0FD127A55E4FE7F0E90A8
:0E1861000017E0FD7C00127A55127B69802F83
:10186F00E490001AF07F017B057A0379C412794E58
:10187F007F027B057A0379D512794E1279EDE4FE5A
:10188F007FC81279D51279ED7E027FBC1279D512FD
:0B189F00063130800C2081093000066B
:1018AA001279ED12634790001AE0B4010280030234
:0218BA001AD240
:1018BC00900017E0B401005003021A2AE0B40A01A8
:0618CC00D34003021A2ABA
:1018D200E0FB24FFFFE434FFFEE4FC7D0A12014139
:1018E200EF2410FFE43E9000BEF0A3EFF0EB2400E3
:1018F200FBE43455FAC002C0039000BEE0FEA3E050
:10190200FF127A83D005D0F0EEB5F00280030219FF
:0A191200E2EFB5050280030219E2BE
:10191C007F017B057A0379E612794E900017E0FB84
:10192C00E4C0E0C0037B027A0079477D057C037834
:10193C00F712081D158115817F027B027A00794709
:10194C0012794E9000BFE02401FF9000BEE03400FD
:10195C00FE127A83EF90000BF09000BFE02402FFA0
:10196C009000BEE03400FE127A83EE900000F0A3EB
:10197C00EFF09000BFE02403FF9000BEE03400FEC7
:10198C00127A83EF900002F09000BFE02404FF90E5
:10199C0000BEE03400FE127A83EE900007F0A3EF55
:1019AC00F09000BFE02405FF9000BEE03400FE1272
:1019BC007A83EE900009F0A3EFF09000BFE02406CC
:1019CC00FF9000BEE03400FE127A83EE90000CF023
:0619DC00A3EFF0021AD295
:1019E2007F017B057A04790912794E7F027B057AA1
:1019F2000379B312794EE490000BF0900000740367
:101A0200F0A374E8F07408A3F09000077403F0A345
:101A120074E8F0A37401F0A374F4F090000C740560
:081A2200F0A37478F0021AD25F
:101A2A007F017B057A04790912794E7F027B057A58
:101A3A000379B312794EE4FE7F10127A83BE5559A8
:031A4A00BF015683
:101A4D00E4FE7F11127A83EF90000BF0E4FE7F121B
:101A5D00127A83EE900000F0A3EFF0E4FE7F1312F4
:101A6D007A83EF900002F0E4FE7F14127A83EE90F9
:101A7D000007F0A3EFF0E4FE7F15127A83EE9000DD
:101A8D0009F0A3EFF0E4FE7F16127A83EE90000CBE
:061A9D00F0A3EFF0802F22
:101AA300E490000BF09000007403F0A374E8F0746A
:101AB30008A3F09000077403F0A374E8F0A3740183
:101AC300F0A374F4F090000C7405F0A37478F09014
:101AD300000BE0B40101D34006740290001BF0E454
:101AE300900033F0900037F0A3F0900034F0D2A9C7
:101AF3001207CA900003E4F0A3F004900010F0C2B0
:101B03000190005FF0E4FDFC900062F090000EE0B5
:101B1300FEA3E0FF121491C004C005C006C0077CF9
:101B23006F7D127E837F3A12112C90003B1200E3EB
:101B3300E4FCFD900013E0FEA3E0FF121491C00447
:101B4300C005C006C0077C6F7D127E837F3A1211E9
:101B53002C90003F1200E3E4FCFD900021E0FEA383
:101B6300E0FF121491C004C005C006C00774CDFC89
:101B730014FDFE743DFF12112C9000431200E37517
:101B8300FD7F75ED7F75DD42D2DE7E037FE812793E
:0D1B9300D51277E61279ED1207F412026602
:101BA000120003127A00EF90005CF090005FE0B446
:101BB000050302274E5014E0146020147003021E27
:101BC000A024FE700302211C023ED3E024F970031E
:0B1BD000022DD8147003023C8980C570
:101BDB00D2B2D2B3D2B490005CE0B4015530015212
:081BEB0090001BE06403602779
:101BF3007401900010F0740590005FF01207CA9012
:101C0300001EE0FBE4900035F0A3EBF0A3E4F0A3A7
:071C1300F0900034F0808620
:101C1A001279C27F017B057A04791A12794E7F0202
:101C2A007B057A04792B12794E1279ED7E077FD0E3
:0A1C3A001279D590005CE0B40209B5
:101C440012026D12620C12000690005CE0B40353A1
:031C54003001500C
:081C570090001BE06402602212
:101C5F00740290005FF01207CA90001EE0FBE49040
:101C6F000035F0A3EBF0A3E4F0A3F0900034F00202
:021C7F003ED352
:101C81001279C27F017B057A04793C12794E7F0279
:101C91007B057A04792B12794E1279ED7E077FD07C
:101CA1001279D5021BA07F05127C65EE90006CF0C5
:0F1CB100A3EFF0900011E0B401028003021D7E4A
:101CC00090000BE0600F14600C14604214603F142D
:051CD0006076021D7E9C
:101CD500E4FCFD90006CE0FEA3E0FF121491C0044B
:101CE500C005C006C007900043121285C004C00598
:101CF500C006C0077455FEFCFD743FFF12112C127F
:101D05001495EF900002F08070E4FCFD90006CE00B
:101D1500FEA3E0FF121491C004C005C006C00790E1
:101D25000043121285C004C005C006C00774ABFC91
:101D350014FDFE743EFF12112C121495EF90000253
:101D4500F08036E4FCFD90006CE0FEA3E0FF121489
:101D550091C004C005C006C007900043121285C09B
:101D650004C005C006C007E4FEFCFD743FFF121168
:101D75002C121495EF900002F0900000E0C0E0A353
:101D8500E0C0E0A3E0FBE4C0E0C0037B027A007999
:101D9500477D057C04784D12081D74FC2581F5816D
:101DA500900002E07006744190004DF07B027A00CD
:101DB500794790000BE0FD1207767F017B027A00E0
:101DC500794712794E900020E0FF127C65EE900075
:101DD500C0F0A3EFF0E4FCFD90006CE0FEA3E0FF93
:101DE500121491C004C005C006C00790004312122A
:101DF50085C004C005C006C0077466FEFCFD743FBF
:0F1E0500FF121522BFFF028006900002E0701945
:101E14007B027A0079477D057C04785E12081D7484
:091E240006900047F0C201806540
:101E2D00E4FCFD9000C0E0FEA3E0FF121491C0049D
:101E3D00C005C006C007900043121285C004C0053E
:101E4D00C006C007E4FCFD90006CE0FEA3E0FF12AD
:101E5D001491C004C005C006C0079000431212853E
:101E6D00C004C005C006C0077B027A0079477D0516
:101E7D007C04786F12081D74F82581F58174029029
:101E8D000047F0D2017F027B027A00794712794E2A
:101E9D00021BA0D2B3D2B41277E67F05127C65E4A3
:101EAD00FCFD121491C004C005C006C0079000438C
:101EBD00121285C004C005C006C0077466FEFCFD85
:091ECD00743FFF121522BFFF4112
:101ED600C201740890005FF0E4A3F07404A3F0124A
:101EE60079ED1277E61207CA7F05127C65EE90003F
:101EF6002BF0A3EFF0900020E0FF127C65EE90003F
:101F06002FF0A3EFF0900035E4F0A37404F0021B69
:101F1600A090005CE0B40307900035E4F0A3F090D5
:061F2600005CE0B4025073
:101F2C007B057A047980123ED6EF64016003023E91
:011F3C00D3D1
:101F3D007F05127C65EE90002BF0A3EFF01277E693
:101F4D001279ED740890005FF0E4A3F07402A3F031
:101F5D001207CA900020E0FF127C65EE90002FF072
:101F6D00A3EFF0900035E4F0A37404F0021BA07B06
:101F7D00027A0079477D057C04789112081D7B0259
:101F8D007A00795290000BE0FD12077674069000EE
:101F9D0047F07F017B027A00794712794E90003528
:101FAD00E0C0E0A3E0C0E07B027A0079477D057CCC
:101FBD000478A212081D158115817402900047F056
:071FCD00900032E0B4010AAC
:0A1FD4007407900048F0C2B28002CA
:101FDE00D2B27F027B027A00794712794E90003599
:0D1FEE00E0600302210EA3E0600302210E5B
:101FFB00C2B275FD0175ED0175DD42D2DE90003F79
:10200B0012009CE4FCFD900009E0FEA3E0FF12141B
:10201B009112112C121495EE900066F0A3EFF09034
:10202B000003E4F0A3F0C0E0C0E07461C0E07445CD
:10203B00C0E0900007E0FEA3E0FFE4FCFD1214916A
:10204B00121288C004C005C006C007E4FCFD74C8AA
:10205B00FE7442FF12112C121495EE900005F0A3A2
:10206B00EFF07B027A0079477D057C0478B3120888
:10207B001D7406900047F07F017B027A00794712AE
:10208B00794E7F027B057A0479C412794E7F011257
:10209B007923900066E0FEA3E0FF7D03126FEBEE69
:1020AB00900064F0A3EFF07F027B057A0479C412F1
:1020BB00794EE4FF127923740490005FF0E49000F2
:0620CB0062F090005BF0E2
:1020D100900064E0FCA3E0FD90005BE0FA2AFB24A1
:1020E10082F582E43400F583ECF0A3EDF090006C0E
:1020F100E0FCA3E0FDEB2496F582E43400F583ECEB
:10210100F0A3EDF090005BE004F0B40AC390003757
:10211100E4F0A3F0900034F0021BA0C2B290005C86
:10212100E064016004E0B403067405900062F0907D
:092131000005E0705DA3E07059A7
:10213A00900004E004F09000037003E004F0E4C0AF
:10214A00E0C0E07461C0E07445C0E0E4FCFD9000CA
:10215A0064E0FEA3E0FF121491C004C005C006C0EB
:10216A000790003F121285121288C004C005C006EB
:10217A00C007E4FCFD74C8FE7442FF12112C12144D
:10218A0095EE900005F0A3EFF090005CE0B4026DCC
:10219A007B057A047980123ED6EF64016003023E21
:0121AA00D361
:1021AB007F05127C65EE90002BF0A3EFF01277E623
:1021BB001279ED740890005FF0E4A3F07402A3F0C1
:1021CB00900003E0FAA3E0FB900027EAF0A3EBF00A
:1021DB00900037E0FAA3E0FB900029EAF0A3EBF0C4
:1021EB00900020E0FF127C65EE90002FF0A3EFF043
:1021FB00900035E4F0A37404F0021BA0900034E0CF
:0D220B00F5F090005DE065F070030223C95E
:10221800900062E0B40001D34003E014F090002085
:10222800E0FF127C65EE9000C0F0A3EFF07F04128F
:1022380076AFEE900092F0A3EFF09000C21200EF9C
:0922480000000000E490005BF0CE
:1022510090005BE025E02484F582E43400F583E01E
:10226100FCA3E0FD90005BE0FA2AFF2482F582E402
:102271003400F583ECF0A3EDF09000C212009CEF66
:102281002482F582E43400F583E0FEA3E0FFE4FC60
:10229100FD12012C9000C21200E390005BE004F0FB
:1022A100B408AD75F0039000C21200D71201179067
:1022B1000064EEF0A3EFF0A3E0FEA3E0FFE4FCFD79
:1022C100121491C004C005C006C0077C0A7DD77EE8
:1022D100A37F3C12112C121495EE90007AF0A3EF1B
:1022E100F0900064E0FCA3E0FDA3E0FAA3E0FB9022
:1022F100007BE0F8EBC398FB90007AE0F8EA98FAEB
:10230100F5F0ECB5F004EDB50300401EE0FAA3E0F2
:10231100FB900067E02BFB900066E03AFAF5F0ECE9
:0A232100B5F005EDB50301D340153A
:10232B00900066E0FEA3E0FF7D04126FEBEE9000E1
:10233B0064F0A3EFF01276EFEE9000A6F0A3EFF0AF
:0F234B009000C21200EF00000000E490005BF071
:10235A0090005BE025E02498F582E43400F583E000
:10236A00FCA3E0FD90005BE0FA2AFF2496F582E4E4
:10237A003400F583ECF0A3EDF09000C212009CEF5C
:10238A002496F582E43400F583E0FEA3E0FFE4FC42
:10239A00FD12012C9000C21200E390005BE004F0F1
:1023AA00B408AD75F0039000C21200D7120117905D
:1023BA00006CEEF0A3EFF0900034E090005DF09036
:1023CA00006CE0B40006A3E0B40001D35003022479
:1023DA00CEE4FCFD90006CE0FEA3E0FF121491C075
:1023EA0004C005C006C007900043121285C004C08D
:1023FA0005C006C007900002E0FB7A00E433E4500F
:10240A000114FCFDAE02AF03121454C004C005C08F
:10241A0006C007E4FCFD900015E0FEA3E0FF1214DD
:10242A0091C004C005C006C0077C6F7D127E837F01
:10243A003A12112C12112C121522BFFF028003022C
:02244A0024CE9E
:10244C0090006CE0FAA3E0FB90002BEAF0A3EBF019
:10245C001277E6900003E0FAA3E0FB900027EAF085
:10246C00A3EBF0900037E0FAA3E0FB900029EAF030
:10247C00A3EBF0900020E0FF127C65EE90002FF0B3
:0A248C00A3EFF090001BE0B4011D67
:10249600900012E0FBE4900035F0A3EBF074059099
:0D24A600005FF0900037E4F0A3F0023ED399
:1024B3001279ED740890005FF0E4A3F004A3F090A8
:1024C3000035E4F0A37404F0021BA0E4FCFD9000CB
:1024D3006CE0FEA3E0FF121491C004C005C006C067
:1024E30007900043121285C004C005C006C00774DC
:0D24F30066FEFCFD743FFF121522BFFF5F67
:102500001279ED1277E6740890005FF0E4A3F0749E
:1025100004A3F0900003E0FAA3E0FB900027EAF0A8
:10252000A3EBF0900037E0FAA3E0FB900029EAF07B
:10253000A3EBF090006CE0FAA3E0FB90002BEAF034
:10254000A3EBF0900020E0FF127C65EE90002FF0EE
:10255000A3EFF0900035E4F0A37404F0021BA09008
:102560000003E0FAA3E0F4FBEAF4FA0BEB70010AD3
:10257000C002C0037B027A0079477D057C0478D5D0
:1025800012081D15811581900010E06401600A9009
:09259000000BE0B40101D340107E
:102599007B027A00794990000BE0FD1207768017DB
:1025A900744490004AF014A3F0743AA3F090001018
:1025B900E0243090004DF0900031E0FA7404C39AA1
:1025C900900047F07406A3F07F017B027A007947F7
:0C25D90012794E900062E060030226EAD6
:1025E500900037E0600302266EA3E0707C90003413
:1025F500E0FBE4C0E0C003FCFD900064E0FEA3E066
:10260500FF121491C004C005C006C00790003F1218
:102615001285C004C005C006C0077C6F7D127E838D
:102625007F3A12112CC004C005C006C007E4FCFDAA
:1026350090006CE0FEA3E0FF121491C004C005C039
:1026450006C007900043121285C004C005C006C02D
:10265500077B027A0079477D057C0478E612081D20
:1026650074F62581F581022740900037E0C0E0A38C
:10267500E0C0E0E4FCFD900064E0FEA3E0FF12147E
:1026850091C004C005C006C00790003F121285C066
:1026950004C005C006C0077C6F7D127E837F3A1299
:1026A500112CC004C005C006C007E4FCFD90006CF9
:1026B500E0FEA3E0FF121491C004C005C006C007E8
:1026C500900043121285C004C005C006C0077B02F6
:1026D5007A0079477D057C0478F912081D74F62582
:0526E50081F581805623
:1026EA00E5FDFF7E00E4FC7D64120141E4FC7DFF10
:1026FA00120155C006C007E4FCFD9000C0E0FEA32D
:10270A00E0FF121491C004C005C006C00790004340
:10271A00121285C004C005C006C0077B027A007980
:10272A00477D057C05780C12081D74FA2581F58110
:10273A007425900056F07F027B027A00794712795D
:10274A004E021BA0D2B2D2B41277E67F05127C6584
:10275A00E4FCFD121491C004C005C006C007900035
:10276A0043121285C004C005C006C0077466FEFC89
:0A277A00FD743FFF121522BFFF415E
:102784001279ED1277E6C201740890005FF0E4A3B9
:10279400F07404A3F090006CE0FAA3E0FB90002B2B
:1027A400EAF0A3EBF0900020E0FF127C65EE9000CD
:1027B4002FF0A3EFF0900035E4F0A37404F0021BB3
:1027C400A090005CE0B40107900035E4F0A3F09021
:0627D400005CE0B4024DC0
:1027DA007B057A05791E123ED6EF64016003023E3C
:0127EA00D31B
:1027EB007F05127C65EE90002BF0A3EFF09000209C
:1027FB00E0FF127C65EE90002FF0A3EFF01277E66E
:10280B001279ED740890005FF0E4A3F07402A3F06A
:10281B00900035E4F0A37404F0021BA07B027A0055
:10282B0079477D057C05782F12081D7B027A00798C
:10283B004F90000BE0FD1207767406900047F07F77
:10284B00017B027A00794712794E900035E0C0E0A7
:10285B00A3E0C0E07B027A0079477D057C0478A277
:10286B0012081D158115817402900047F0900032FB
:04287B00E0B4010ABA
:0A287F007407900048F0C2B3800215
:10288900D2B37F027B027A00794712794E900035E4
:0D289900E06003022DCAA3E06003022DCA17
:1028A60090003B12009CE4FCFD74A0FE7441FF12F4
:1028B600112C121495EE900070F0A3EFF0E4FCFDDD
:1028C600900018E0FEA3E0FF121491C004C005C0FA
:1028D60006C0077C6F7D127E837F3A12112CC004DE
:1028E600C005C006C007900002E0FF7E00E433E4A6
:1028F600500114FCFD12145412112CC004C005C062
:1029060006C007900043121129121495EE90007428
:10291600F0A3EFF090000BE0705D90001CE0FF7EEE
:1029260000E433E4500114FCFD121454C004C00545
:10293600C006C0077C6F7D127E837F3A12112CC0C1
:1029460004C005C006C007900043121129C004C088
:1029560005C006C007900002E0FDFFE4FE33E45028
:102966000114FDFC12145412112C121495EE900051
:1029760076F0A3EFF0806490001DE0FBE433E450B2
:102986000114FCFD7E00AF03121454C004C005C040
:1029960006C0077C6F7D127E837F3A12112CC0041D
:1029A600C005C006C007900043121129C004C00527
:1029B600C006C007900002E0FD7C00E4C0E0EDFF29
:1029C600D0E0FE33E4500114FDFC12145412112C15
:1029D600121495EE900076F0A3EFF090000CE0FE56
:1029E600A3E0FFE4FCFD121491C004C005C006C0BC
:1029F600077C6F7D127E837F3A12112CC004C005BE
:102A0600C006C007900002E0FD7C00E4C0E0EDFFD8
:102A1600D0E0FE33E4500114FDFC12145412112CC4
:102A2600C004C005C006C007900043121129121445
:102A360095EE90006AF0A3EFF0900000E0FEA3E0B0
:102A4600FF900007E0FCA3E0FD12017DE4FCFD120F
:102A56001491C004C005C006C007749AFC14FDFE9C
:102A6600743FFF12112CC004C005C006C007E4FC69
:102A7600FD7461FE7445FF12112C121495EE900040
:102A860039F0A3EFF0900002E0FF7E00E433E4505B
:102A96000114FCFD121454C004C005C006C0077C16
:102AA600EC7D517EB87F3F12112CC004C005C006D4
:102AB600C007900043121129121495EE900078F089
:102AC600A3EFF090004312009CE4FEFCFD743FFF70
:102AD60012112C121495EE90007CF0A3EFF09000EA
:102AE6004312009C7C0A7DD77E237F3C12112C1258
:102AF6001495EE900080F0A3EFF0900020E0B4046F
:102B06006DE4FCFD90000CE0FEA3E0FF121491C002
:102B160004C005C006C0077C6F7D127E837F3A1213
:102B2600112CC004C005C006C007900002E0FF7E5D
:102B360000E433E4500114FCFD12145412112CC0AD
:102B460004C005C006C007E4FCFD74C0FE743FFF68
:102B5600120FD5C004C005C006C00790004312116D
:102B660029121495EE90006EF0A3EFF0801D9000F0
:102B76004312009CE4FCFD7428FE7441FF12112CE4
:102B8600121495EE90006EF0A3EFF090000BE0FAB1
:102B960064026003BA032D90003B12009C90000271
:102BA600E0FF7E00E4FC7D50120141EE33E450016B
:102BB60014FDFC12145412112C121495EE9000728E
:102BC600F0A3EFF090000BE0B4043A900000E4FCB0
:102BD600FDE0FEA3E0FF121491C004C005C006C0CC
:102BE600077C297D5C7E8F7F3D12112CC004C005B9
:102BF600C006C00790003B121129121495EE9000F2
:102C060072F0A3EFF090000BE0B40101D3404BE467
:102C1600FCFD900072E0FEA3E0FF121491C004C018
:032C260005C006E0
:102C2900C00790003B12009CE4FCFD74A0FE7442B6
:102C3900FF12112C121522BFFF1D90003B12009CA0
:102C4900E4FCFD74A0FE7442FF12112C121495EEDF
:102C5900900072F0A3EFF090000BE0B40101D340B3
:102C6900067401900010F0C202E490005EF090003A
:102C790060F090006CE0FAA3E0FB900068EAF0A332
:102C8900EBF0E4900062F090007EF0A3F090006316
:102C9900F0900003F0A3F0C0E0C0E07461C0E074FC
:102CA90045C0E0900007E0FAA3E0FBE4FCFDAE02BA
:102CB900AF03121491121288C004C005C006C007E0
:102CC900E4FCFD74C8FE7442FF12112C121495EE37
:102CD900900005F0A3EFF0C2B375FE0175EE017522
:102CE900DE42D2DEC20390003B12009CE4FCFD9060
:102CF9000007E0FEA3E0FF12149112112C121495A3
:102D0900EE900066F0A3EFF07B027A0079477D052B
:102D19007C05784112081D7406900047F07F017BFD
:102D2900027A00794712794E7F027B057A0479C4C9
:102D390012794E7F01127923900066E0FEA3E0FF2D
:102D49007D06126FEBEE900064F0A3EFF07F027B3B
:102D5900057A0479C412794EE4FF127923E49000CC
:022D69005BF01D
:102D6B00900064E0FCA3E0FD90005BE0FA2AFB24FA
:102D7B0082F582E43400F583ECF0A3EDF090006C67
:102D8B00E0FCA3E0FDEB2496F582E43400F583EC44
:102D9B00F0A3EDF0900020E0FF127C6590005BE06B
:102DAB00FA2A24AAF582E43400F583EEF0A3EFF0BF
:102DBB0090005BE004F0B40AA7740790005FF090FA
:102DCB000037E4F0A3F0900034F0021BA0C2B390E4
:102DDB00005CE064016004E0B403067405900062DB
:0B2DEB00F0900005E0705DA3E070595F
:102DF600900004E004F09000037003E004F0E4C0E7
:102E0600E0C0E07461C0E07445C0E0E4FCFD900001
:102E160064E0FEA3E0FF121491C004C005C006C022
:102E26000790003B121285121288C004C005C00626
:102E3600C007E4FCFD74C8FE7442FF12112C121484
:102E460095EE900005F0A3EFF0900039E0706EA3C8
:032E5600E0706ABF
:102E59001277E61279ED740890005FF0E4A3F0A30D
:102E6900F0900003E0FAA3E0FB900023EAF0A3EB63
:102E7900F0900037E0FAA3E0FB900025EAF0A3EB1D
:102E8900F090006CE0FAA3E0FB90002BEAF0A3EBD2
:102E9900F090007EE0FAA3E0FB90002DEAF0A3EBAE
:102EA900F0900020E0FF127C65EE90002FF0A3EF78
:102EB900F0900035E4F0A37404F090005CE0B402F3
:062EC900028003022F52FB
:0E2ECF007B057A05791E123ED6EF6401707500
:102EDD001277E61279ED7401900010F074089000ED
:102EED005FF0E4A3F07402A3F0900003E0FAA3E016
:102EFD00FB900023EAF0A3EBF0900037E0FAA3E09B
:102F0D00FB900025EAF0A3EBF090006CE0FAA3E053
:102F1D00FB90002BEAF0A3EBF090007EE0FAA3E02B
:102F2D00FB90002DEAF0A3EBF0900020E0FF127C67
:102F3D0065EE90002FF0A3EFF0900035E4F0A37450
:0B2F4D0004F0021BA030030302310D52
:102F5800900034E0F5F090005DE065F07003023217
:012F6800E880
:102F6900900062E0B40001D34003E014F07F07123F
:102F790076AFEE900092F0A3EFF09000C21200EF4E
:092F890000000000E490005BF080
:102F920090005BE025E02484F582E43400F583E0D0
:102FA200FCA3E0FD90005BE0FA2AFF2482F582E4B4
:102FB2003400F583ECF0A3EDF09000C212009CEF18
:102FC2002482F582E43400F583E0FEA3E0FFE4FC12
:102FD200FD12012C9000C21200E390005BE004F0AD
:102FE200B408AD75F0039000C21200D71201179019
:102FF2000064EEF0A3EFF0A3E0FEA3E0FFE4FCFD2B
:10300200121491C004C005C006C0077C0A7DD77E99
:10301200A37F3C12112C121495EE90007AF0A3EFCC
:10302200F0900064E0FCA3E0FDA3E0FAA3E0FB90D3
:10303200007BE0F8EBC398FB90007AE0F8EA98FA9C
:10304200F5F0ECB5F004EDB50300401EE0FAA3E0A4
:10305200FB900067E02BFB900066E03AFAF5F0EC9B
:0A306200B5F005EDB50301D34015EC
:10306C00900066E0FEA3E0FF7D07126FEBEE900090
:10307C0064F0A3EFF01276EFEE9000A6F0A3EFF061
:0F308C009000C21200EF00000000E490005BF023
:10309B0090005BE025E02498F582E43400F583E0B2
:1030AB00FCA3E0FD90005BE0FA2AFF2496F582E496
:1030BB003400F583ECF0A3EDF09000C212009CEF0E
:1030CB002496F582E43400F583E0FEA3E0FFE4FCF4
:1030DB00FD12012C9000C21200E390005BE004F0A3
:1030EB00B408AD75F0039000C21200D7120117900F
:1030FB00006CEEF0A3EFF0900034E090005DF00276
:02310B0032E8A8
:10310D00900034E0F5F090005DE065F07003023260
:01311D00E8C9
:10311E00900062E0B40001D34003E014F01276EFA9
:10312E00EE9000A6F0A3EFF09000C21200EF0000A8
:07313E000000E490005BF0CB
:1031450090005BE025E02498F582E43400F583E007
:10315500FEA3E0FF90005BE0FA2AFD7C002496F5D3
:1031650082E43400F583EEF0A3EFF09000C2120084
:103175009CED2496F582E43400F583E0FEA3E0FFA0
:10318500E4FD12012C9000C21200E390005BE00404
:10319500F0B408AC75F0039000C21200D712011705
:1031A50090006CEEF0A3EFF090000BE0B4042EE479
:1031B500FCFD90006AE0FEA3E0FF121491C004C07C
:1031C50005C006C0077C0A7DD77EA37F3C12112C63
:1031D500121495EE90007AF0A3EFF0801C90004356
:1031E50012009C7C0A7DD77EA37F3B12112C121402
:1031F50095EE90007AF0A3EFF090006CE0FCA3E070
:10320500FD90006AE0FAA3E0FB90007BE0F8EBC3D9
:1032150098FB90007AE0F8EA98FAF5F0ECB5F0043E
:10322500EDB50300401EE0FAA3E0FB90006BE02B38
:10323500FB90006AE03AFAF5F0ECB5F005EDB50360
:0432450001D340135E
:1032490090006AE0FEA3E0FF127512EE90006CF0A8
:10325900A3EFF07F071276AFEE900092F0A3EFF0A4
:0F3269009000C21200EF00000000E490005BF044
:1032780090005BE025E02484F582E43400F583E0E7
:10328800FEA3E0FF90005BE0FA2AFD7C002482F5B3
:1032980082E43400F583EEF0A3EFF09000C2120050
:1032A8009CED2482F582E43400F583E0FEA3E0FF80
:1032B800E4FD12012C9000C21200E390005BE004D0
:1032C800F0B408AC75F0039000C21200D7120117D1
:1032D800900064EEF0A3EFF0900034E090005DF011
:1032E80090000BE06009E0B401028003023395907E
:1032F8000070E0FAF5F0A3E0FB900064E0B5F0069A
:0B330800A3E0B50301D340030233959E
:103313007F05127C65EE90002BF0A3EFF01277E6A9
:1033230075FD7F75ED7F75DD42D2DE1279ED740197
:10333300900010F0C201740890005FF0E4A3F074F1
:1033430004A3F0900003E0FAA3E0FB900023EAF06B
:10335300A3EBF0900037E0FAA3E0FB900025EAF03E
:10336300A3EBF090007EE0FAA3E0FB90002DEAF0DF
:10337300A3EBF0900020E0FF127C65EE90002FF0AD
:10338300A3EFF0900035E4F0A37404F01277E602A3
:103393001BA090000BE0FAB40101D3500302346B7D
:1033A300900070E0FCA3E0FD900064E0B50406A388
:1033B300E0B50501D3400302346B90006CE0FEA33B
:1033C300E0FF90007CE0FCA3E0FD90006BE02DFDAE
:1033D30090006AE03CFCF5F0EEB5F005EFB50501B1
:0633E300D3500302346B1D
:1033E9007F05127C65EE90002BF0A3EFF01277E6D3
:1033F90075FD7F75ED7F75DD42D2DE1279ED7401C1
:10340900900010F0C201740890005FF0E4A3F0741A
:1034190004A3F0900003E0FAA3E0FB900023EAF094
:10342900A3EBF0900037E0FAA3E0FB900025EAF067
:10343900A3EBF090007EE0FAA3E0FB90002DEAF008
:10344900A3EBF0900020E0FF127C65EE90002FF0D6
:10345900A3EFF0900035E4F0A37404F01277E602CC
:103469001BA090000BE06009E0B401028003023563
:013479000D45
:10347A00900074E0FAA3E0FB90006CE0B50206A3AA
:07348A00E0B50301D3407718
:0C34910090005EE004F0B40401D3407031
:10349D007F05127C65EE90002BF0A3EFF01277E61E
:1034AD001279ED740890005FF0E4A3F07403A3F0BB
:1034BD00900003E0FAA3E0FB900023EAF0A3EBF009
:1034CD00900037E0FAA3E0FB900025EAF0A3EBF0C3
:1034DD0090007EE0FAA3E0FB90002DEAF0A3EBF064
:1034ED00900020E0FF127C65EE90002FF0A3EFF02E
:0B34FD00900035E4F0A37404F080059B
:10350800E490005EF090000BE06009E0B4010280F6
:10351800030236C2900078E0FAA3E0FB90006CE06A
:0E352800B50206A3E0B50301D350030236C27C
:1035360090007EE0FAA3E0FB90006CE0B50206A3E3
:07354600E0B50301D3401EB4
:10354D0090006CE0FAA3E0FB90007EEAF0A3EBF0B4
:0E355D0090000BE060030236C2C2020236C2CA
:10356B00900077E0FB900076E0C313CB13CBFA907F
:10357B00007EE0FCA3E0FD90006DE0F8EDC398FD4C
:10358B0090006CE0F8EC98B50205EDB50301D34063
:10359B0002D202900076E0FCA3E0FD90007EE0FA00
:1035AB00A3E0FB90006DE0F8EBC398FB90006CE0A0
:1035BB00F8EA98B50405EBB50501D350030236C202
:0D35CB00900010E0B40101D3500302365807
:1035D800E014F0740290005FF01277E6900027E4A0
:1035E800F0A3F0A3F0A3F0900003E0FAA3E0FB90AF
:1035F8000023EAF0A3EBF0900037E0FAA3E0FB9099
:103608000025EAF0A3EBF090006CE0FAA3E0FB9051
:10361800002BEAF0A3EBF090007EE0FAA3E0FB9029
:10362800002DEAF0A3EBF0900020E0FF127C65EE9D
:1036380090002FF0A3EFF0900012E0FBE49000352B
:10364800F0A3EBF0A3E4F0A3F0900034F0021BA089
:103658001277E61279ED740890005FF0E4A3F0A306
:10366800F0900003E0FAA3E0FB900023EAF0A3EB5C
:10367800F0900037E0FAA3E0FB900025EAF0A3EB16
:10368800F090006CE0FAA3E0FB90002BEAF0A3EBCB
:10369800F090007EE0FAA3E0FB90002DEAF0A3EBA7
:1036A800F0900020E0FF127C65EE90002FF0A3EF71
:1036B800F0900035E4F0A37404F090000BE0FAB445
:1036C80001028003023866900078E0FCF5F0A3E080
:1036D800FD90006CE0B5F006A3E0B50501D35003FA
:0336E8000238663F
:1036EB00900035E06003023866A3E06003023866A1
:1036FB00900080E0C0E0A3E0C0E0900068E0FAA397
:10370B00E0FB90006DE0F8EBC398FF90006CE0F8E5
:10371B00EA98FE120212D003D0F0EEB5F004EFB52A
:07372B0003004003023846D1
:10373200900060E004F0B40101D34002D202900094
:0B37420060E0B40401D3500302384DD6
:0D374D00900010E0B40101D350030237DA00
:10375A00E014F0740290005FF01277E6900027E41C
:10376A00F0A3F0A3F0A3F0900003E0FAA3E0FB902B
:10377A000023EAF0A3EBF0900037E0FAA3E0FB9015
:10378A000025EAF0A3EBF090006CE0FAA3E0FB90CE
:10379A00002BEAF0A3EBF090007EE0FAA3E0FB90A6
:1037AA00002DEAF0A3EBF0900020E0FF127C65EE1A
:1037BA0090002FF0A3EFF0900012E0FBE4900035A8
:1037CA00F0A3EBF0A3E4F0A3F0900034F0021BA006
:1037DA001277E61279ED740890005FF0E4A3F0A383
:1037EA00F0900003E0FAA3E0FB900023EAF0A3EBD9
:1037FA00F0900037E0FAA3E0FB900025EAF0A3EB93
:10380A00F090006CE0FAA3E0FB90002BEAF0A3EB47
:10381A00F090007EE0FAA3E0FB90002DEAF0A3EB23
:10382A00F0900020E0FF127C65EE90002FF0A3EFED
:0C383A00F0900035E4F0A37404F0800767
:10384600C202E4900060F0900035E4F0A3743CF00E
:1038560090006CE0FAA3E0FB900068EAF0A3EBF0BE
:0D38660090000BE0B40101D3500302397053
:1038730090006AE0FAA3E0FBA3E0B50205A3E0B57C
:0738830003004018200315AB
:10388A00D202D20390003AE02410FB900039E034CF
:10389A000EF0A3EBF0900072E0FAA3E0FB90006454
:1038AA00E0B50205A3E0B503004003023970200326
:1038BA0003023970900070E0FAA3E0FB900064E024
:1038CA00B50206A3E0B50301D35003023970900094
:1038DA006CE0FCA3E0FD90007CE0FAA3E0FB900022
:1038EA006BE02BFB90006AE03AFAF5F0ECB5F004D5
:0638FA00EDB50300507063
:103900007401900010F01277E61279ED74089000BF
:103910005FF0E4A3F0A3F0900003E0FAA3E0FB90D3
:103920000023EAF0A3EBF0900037E0FAA3E0FB906D
:103930000025EAF0A3EBF090006CE0FAA3E0FB9026
:10394000002BEAF0A3EBF090007EE0FAA3E0FB90FE
:10395000002DEAF0A3EBF0900020E0FF127C65EE72
:1039600090002FF0A3EFF0900035E4F0A37404F082
:103970009000C21200EF00000000900020E0FF1253
:0F3980007C65EE9000BAF0A3EFF0E490005BF0EE
:10398F0090005BE025E024ACF582E43400F583E0A1
:10399F00FEA3E0FF90005BE0FA2AFD7C0024AAF56D
:1039AF0082E43400F583EEF0A3EFF09000C2120032
:1039BF009CED24AAF582E43400F583E0FEA3E0FF3A
:1039CF00E4FD12012C9000C21200E390005BE004B2
:1039DF00F0B408AC75F0039000C21200D7120117B3
:1039EF009000C0EEF0A3EFF090006EE0F5F0A3E0D2
:1039FF00FB9000C0E0B5F005A3E0B5030040030263
:023A0F003A91EA
:0C3A1100900063E004F0B40401D340799D
:103A1D001277E61279ED7401900010F074089000A1
:103A2D005FF0E4A3F07405A3F0900035E4F0A37407
:103A3D0004F0900003E0FAA3E0FB900023EAF0A36A
:103A4D00EBF0900037E0FAA3E0FB900025EAF0A33D
:103A5D00EBF090006CE0FAA3E0FB90002BEAF0A3F2
:103A6D00EBF090007EE0FAA3E0FB90002DEAF0A3CE
:103A7D00EBF09000C0E0FAA3E0FB90002FEAF0A37A
:043A8D00EBF08005D5
:103A9100E4900063F0900003E0C0E0A3E0C0E07BAD
:103AA100027A0079477D057C0478D512081D1581BD
:103AB1001581900010E06401600A90000BE0B401F0
:043AC10001D34010DD
:103AC5007B027A00794990000BE0FD12077680179A
:103AD500744390004AF004A3F0743AA3F0900010E8
:0A3AE500E0243090004DF020020AAA
:0A3AEF00900031E0900047F0800DD8
:103AF900900032E0B401067404900047F074059018
:103B09000048F07F017B027A00794712794E9000D4
:073B190062E06003023C259D
:103B2000900037E06003023BA9A3E0707C90003472
:103B3000E0FBE4C0E0C003FCFD900064E0FEA3E015
:103B4000FF121491C004C005C006C00790003B12CC
:103B50001285C004C005C006C0077C6F7D127E833D
:103B60007F3A12112CC004C005C006C007E4FCFD5A
:103B700090006CE0FEA3E0FF121491C004C005C0E9
:103B800006C007900043121285C004C005C006C0DD
:103B9000077B027A0079477D057C0478E612081DD0
:103BA00074F62581F581023C7B900037E0C0E0A3EC
:103BB000E0C0E0E4FCFD900064E0FEA3E0FF12142E
:103BC00091C004C005C006C00790003B121285C01A
:103BD00004C005C006C0077C6F7D127E837F3A1249
:103BE000112CC004C005C006C007E4FCFD90006CA9
:103BF000E0FEA3E0FF121491C004C005C006C00798
:103C0000900043121285C004C005C006C0077B02A5
:103C10007A0079477D057C0478F912081D74F62531
:053C200081F5818056D2
:103C2500E5FEFF7E00E4FC7D64120141E4FC7DFFBE
:103C3500120155C006C007E4FCFD9000C0E0FEA3DC
:103C4500E0FF121491C004C005C006C007900043F0
:103C5500121285C004C005C006C0077B027A007930
:103C6500477D057C05780C12081D74FA2581F581C0
:103C75007425900056F07F027B027A00794712790D
:103C85004E021BA0D2B2D2B3900061E0B403028011
:103C950050500BE06012146022146032807AE024E8
:083CA500FC60511460618070A5
:103CAD007B027A0079477D057C05785212081DD27A
:103CBD00B4805D7B027A0079477D057C05786312BF
:103CCD00081DD2B4804A7B027A0079477D057C05B8
:103CDD00787412081DC2B480377B027A0079477D53
:103CED00057C05788512081DC2B480247B027A00FC
:103CFD0079477D057C05789612081DC2B480117B2D
:103D0D00027A0079477D057C0578A712081DC2B49B
:103D1D007406900047F07F017B027A007947127993
:103D2D004E900035E0FAA3E0FBBA0004B40401D3D1
:103D3D004009900035E4F0A37404F0900035E07074
:053D4D001EA3E0701A46
:103D520012799E900035E4F0A37404F0900060E0C4
:103D620004F0B40501D34002E4F0900060E0B40333
:103D720003023E00500CE0601A14604214605F02BD
:103D82003EB8E024FC7003023E20147003023E7F22
:033D9200023EB836
:103D9500900028E0F4FB900027E0F4FA0BEB7001AB
:103DA5000AC002C0037B027A0079477D057C05784D
:103DB500B812081D15811581023EB8900029E0C092
:103DC500E0A3E0C0E07B027A0079477D057C0578B9
:103DD500C912081D15811581023EB8900023E0C067
:103DE500E0A3E0C0E07B027A0079477D057C057899
:103DF500DA12081D15811581023EB8900025E0C034
:103E0500E0A3E0C0E07B027A0079477D057C057878
:103E1500EB12081D15811581023EB8E4FCFD9000EA
:103E25002BE0FEA3E0FF121491C004C005C006C03C
:103E350007900043121285C004C005C006C007E400
:103E4500FCFD90002DE0FEA3E0FF121491C004C01C
:103E550005C006C007900043121285C004C005C006
:103E650006C0077B027A0079477D057C0578FC1240
:103E7500081D74F82581F5818039E4FCFD90002F3B
:103E8500E0FEA3E0FF121491C004C005C006C00700
:103E9500900043121285C004C005C006C0077B020E
:103EA5007A0079477D057C06780E12081D74FC257D
:103EB50081F5817F027B027A00794712794E900065
:053EC5005CE0B40209FD
:0C3ECA001207F4740190005FF0021BA0CE
:103ED6008B2F8A3089311207F474199000DAF0902A
:103EE6000032E024FF92047F01AB2FAA30A93112E1
:103EF600794E7B027A0079C67D057C067820120809
:103F06001D74069000C8F0E49000DBF0A3F090006A
:063F1600DCE064026078AB
:103F1C00120003127A00EF9000DCF064016004E000
:033F2C00B40329B2
:073F2F009000DBE0B401107B
:103F3600E4F074069000C8F074209000CFF0801270
:103F460074019000DBF074209000C8F074069000B5
:103F5600CFF07F027B027A0079C612794E9000324A
:103F6600E0B4010874079000D5F080067420900034
:0E3F7600D5F0A204E433FA900032E06A6090C5
:103F8400E024FF92049000DAE014F07083E4FF224E
:063F94009000DBE0FF22BB
:103F9A00424154544552592054595045202020201A
:103FAA00003A4E694344202020202020202020204F
:103FBA0020003A4E694D4820202020202020202031
:103FCA002020003A4C69506F2020202020202020F9
:103FDA00202020003A4C69494F4E202020202020E2
:103FEA0020202020003A534C41202020202020204D
:103FFA002020202020004241545445525920434554
:10400A004C4C20202020003A4155544F204445541E
:10401A0045435420202020003A25326420202020C5
:10402A0020202020202020202000424154542E20ED
:10403A0043415041434954592020003A2534646D84
:10404A004168202020202020202000434841524758
:10405A00452043555252454E542020003A25346497
:10406A006D41202020202020202020004449534355
:10407A00482E2043555252454E5420200045584957
:10408A0054204241545445525920202020004E6960
:10409A0043442025326443202534646D4168004E30
:1040AA00694D482025326443202534646D416800F7
:1040BA004C69506F202025316443202534646D41BA
:1040CA0068004C69494F4E202531644320253464E9
:1040DA006D416800534C412020202531644320253E
:1040EA0034646D416800534554204241545445524A
:1040FA0059205459504500204E694344202020201D
:10410A002020202020202000204E694D48202020F9
:10411A00202020202020202000204C69506F2020C1
:10412A0020202020202020202000204C69494F4EAA
:10413A00202020202020202020200020534C412015
:10414A0020202020202020202020200053455420F9
:10415A00424154544552592043454C4C0020253283
:10416A0064202020202020202020202020200053EE
:10417A0045542043415041434954592020202000AE
:10418A00202534646D416820202020202020200032
:10419A00202534646D41202020202020202020006A
:1041AA004C4F41442046524F4D204C4F432E25320E
:1041BA0064005341564520544F204C4F432E202033
:1041CA00253264004552415345204441544120411F
:1041DA005420253264004C6F6164696E6720426125
:1041EA007474657279200046726F6D204C6F63613A
:1041FA0074696F6E2025326400204E6F204261740C
:10420A0074657279204461746100204174204C6F96
:10421A00636174696F6E2025326420004F564552DF
:10422A00575249544520444154413F20002053618C
:10423A0076696E6720426174746572792000205431
:10424A006F204C6F636174696F6E202532642000A1
:10425A00455241534520444154413F2020202020CB
:10426A000045726173696E67204261747465727980
:10427A0020002045584954204D454D4F5259202081
:10428A00202000204E6943442025326443202534EF
:10429A00646D416800204E694D48202532644320F0
:1042AA002534646D416800204C69506F2020253107
:1042BA006443202534646D416800204C69494F4E9F
:1042CA002025316443202534646D41680020534C15
:1042DA004120202025316443202534646D41680043
:1042EA0020454D50545920202020202020202020D5
:1042FA0000202020202020202020202020202020D4
:10430A002000455241534520414C4C2044415441E0
:10431A003F200045726173696E6720416C6C2044CE
:10432A006174610020202046726F6D204D656D6FAB
:10433A0072792020005345542043454C4C53204465
:10434A00455445435400204155544F2020202020F5
:10435A0020202020202000204D414E55414C202075
:10436A002020202020202000534554204348415239
:10437A00474552204D4F444500204359434C452060
:10438A004348415247452020200020434841524794
:0B439A0045204F4E4C592020202000F1
:1043A50020444953434841524745204F4E4C5920DC
:1043B5000053455420434841524745204359434CF7
:1043C500450053455420534F554E4420564F4C55A8
:1043D5004D4500204F4E2020202020202020202049
:1043E50020202000204F464620202020202020206D
:1043F500202020200020202A2A204552524F5220DA
:104405002A2A2020200020204D656D6F72792046D4
:1044150061696C20202000204C4F41442020202041
:104425002053415645202000205341564520202049
:1044350020204552415345200020455241534520F7
:10444500202020464F524D41540020464F524D41A9
:1044550054202020455849542020002045584954CF
:1044650020202020204C4F414420200055736520FA
:104475003C3E20746F2053656C65637400204E6F5D
:1044850074204170706C696361626C652000466FD1
:1044950072205468697320426174746572790020D2
:1044A500466F722054686973204D6F646520200043
:1044B5002043454C4C5320444554454354494F4EA5
:1044C500003A4155544F2020202020202020202034
:1044D50020003A4D414E55414C20202020202020DF
:1044E5002020002043484152474552204D4F444526
:1044F500202020003A4359434C4520434841524728
:1045050045202020003A434841524745204F4E4C14
:104515005920202020003A444953434841524745F9
:10452500204F4E4C592000204348415247452043D7
:1045350059434C45202020003A4E6F74204170703D
:104545006C696361626C65200020534F554E4420B1
:10455500564F4C554D45202020003A4F4E202020E7
:1045650020202020202020202020003A4F464620D1
:1045750020202020202020202020200020455849D0
:1045850054204F5054494F4E532020200020424183
:10459500545445525920204D454D4F525900204DF8
:1045A500454D4F525920204F5054494F4E530020EE
:1045B5004F5054494F4E5320202020455849540010
:1045C50020455849542020202042415454455259F1
:1045D500002020534D4152542043484152474552F3
:1045E5002000202053455256494345204D4F444510
:1045F500202000202020204649524D574152452079
:1046050020202000202056455253494F4E20312E60
:10461500313420200020444953434820432D53542E
:104625004550202020003A253464202020202020D9
:104635002020202020002043555252454E5420531F
:1046450054455020202000205354415254204445C5
:104655004C415920202020003A25336420536563BE
:104665006F6E647320202020002044495343482D59
:104675004348472044454C415900204D41582E2080
:10468500564F4C542F43454C4C20003A25352E327D
:1046950066562020202020202020202000204D4963
:1046A5004E2E20564F4C542F43454C4C2000204E47
:1046B5006943442053454E53495449564520003AD1
:1046C500253264206D562F43656C6C2020202020F8
:1046D5002000204E694D482053454E5349544956B4
:1046E50045200020535550504C59204D4F4E4954AC
:1046F5004F5220003A43482531642020202025359B
:104705002E32665673200020564F4C5441474520A3
:1047150053544550202020003A2534642020202081
:1047250025352E32665620002045584954205345DC
:1047350052564943452020200053455420444953AF
:10474500434820432D535445500053455420435569
:104755005252454E5420535445500053455420530E
:10476500544152542044454C41592000534554204E
:1047750044495343482D4348415247450053455406
:10478500204D41582E20562F43454C4C20003A25AC
:0F479500352E32665620202020202020202000A4
:1047A400534554204D494E2E20562F43454C4C2002
:1047B400004E6943442053454E53495449564520BD
:1047C40020003A2532646D5620202020202020200D
:1047D400202020004E694D482053454E53495449EA
:1047E400564520200053455420535550504C5920D1
:1047F4004D4F4E2E200053455420564F4C544147A4
:07480400452053544550000C
:08480B00C2057524011207F437
:10481300127A008F25E52514600B14601914603695
:05482300146043804415
:10482800E524B40101D3400415248038752406809A
:0648380033E524B406067E
:06483E001207F4E4FF2262
:10484400AF24124BA68F26E526B404037F0422303E
:104854000516E4FF22E524B406005004052480086C
:1048640075240180037F0422E524B404030249C3B0
:104874005014E52414602114700302491B147003BE
:1048840002497E024BA3E52424FB7003024A081468
:084894007003024A750248138B
:10489C007B027A0079DE7D057C3F789A12081D7FB9
:1048AC00017B027A0079DE12794E90000BE0700BDE
:1048BC007F027B057A3F79AB12794E90000BE0FAC0
:1048CC00B4010B7F027B057A3F79BC12794E9000C4
:1048DC000BE0FAB4020B7F027B057A3F79CD12799B
:1048EC004E90000BE0FAB4030B7F027B057A3F7904
:1048FC00DE12794E90000BE0FAB404028003024BF6
:10490C00A37F027B057A3F79EF12794E0248137B25
:10491C00027A0079DE7D057C40780012081D7F014B
:10492C007B027A0079DE12794E900002E0600790EB
:10493C000011E0B401117B027A0079DE7D057C4028
:10494C00781112081D801D900002E0FDE4C0E0C04B
:10495C00057B027A0079DE7D057C40782212081DE9
:10496C00158115817F027B027A0079DE12794E0265
:10497C0048137B027A0079DE7D057C40783412087E
:10498C001D7F017B027A0079DE12794E900000E0E7
:10499C00C0E0A3E0C0E07B027A0079DE7D057C40BC
:1049AC00784512081D158115817F027B027A0079EA
:1049BC00DE12794E0248137B027A0079DE7D057C8B
:1049CC0040785512081D7F017B027A0079DE12793E
:1049DC004E900007E0C0E0A3E0C0E07B027A0079D3
:1049EC00DE7D057C40786612081D158115817F02DD
:1049FC007B027A0079DE12794E02481390000BE0AC
:0E4A0C00FA64026009EA64036004EAB4041666
:104A1A00E525B401021524E525B403028003024BFF
:104A2A00A305240248137B027A0079DE7D057C40C7
:104A3A00787612081D7F017B027A0079DE12794EA0
:104A4A00900009E0C0E0A3E0C0E07B027A0079DED2
:104A5A007D057C40786612081D158115817F027BD1
:104A6A00027A0079DE12794E0248137B027A0079C3
:104A7A00DE7D057C40788712081D7F017B027A0063
:104A8A0079DE12794E90000BE0601514603E1460D6
:104A9A0067147003024B2D147003024B58024B81AA
:104AAA00900000E0C0E0A3E0C0E0900002E0FDE476
:104ABA00C0E0C0057B027A0079DE7D057C407898EB
:104ACA0012081D74FC2581F581024B81900000E0DB
:104ADA00C0E0A3E0C0E0900002E0FDE4C0E0C00551
:104AEA007B027A0079DE7D057C4078A912081D7464
:104AFA00FC2581F581024B81900000E0C0E0A3E033
:104B0A00C0E0900002E0FDE4C0E0C0057B027A004C
:104B1A0079DE7D057C4078BA12081D74FC2581F582
:104B2A00818054900000E0C0E0A3E0C0E090000261
:104B3A00E0FDE4C0E0C0057B027A0079DE7D057CF9
:104B4A004078CC12081D74FC2581F58180299000DB
:104B5A0000E0C0E0A3E0C0E0900002E0FDE4C0E0B5
:104B6A00C0057B027A0079DE7D057C4078DE12087A
:104B7A001D74FC2581F581900002E0600790001108
:044B8A00E0B4010A88
:104B8E0074209000E3F07441A3F07F027B027A0060
:084B9E0079DE12794E02481382
:054BA6008F271207F447
:104BAB0090000BE0600E14600B14602B1460281443
:044BBB006048806767
:104BBF0090000C7405F0A37478F0740190001BF052
:104BCF0075280C75290F752AA0752B07752CD0F534
:104BDF002D804490000C7410F0A37468F074029050
:104BEF00001BF075280375290F752AA0E4F52BF526
:104BFF002C752D01802190000C7409F0A37492F094
:104C0F00740290001BF075280675291B752A58E44D
:104C1F00F52BF52C752D03127A008F2EE52EB4048B
:104C2F0003AF2E22E52714601B147003024EDD1410
:104C3F007003024F4D14700302509414700302510D
:044C4F0056024BAB13
:104C53007F017B057A4079F012794EE52EB4011578
:104C630090000BE0B40001D34005E014F08006741B
:0F4C73000490000BF0E52EB402028003024E41C4
:104C8200900000E0FAA3E0FB900007EAF0A3EBF04B
:104C9200900007E0B40005A3E0B46400500990005E
:104CA20007E4F0A37464F0900007E0FEA3E0FFE4E1
:104CB200FC7D6412017DEE900007F0A3EFF09000FE
:104CC20007E0FEA3E0FFE4FC7D64120141EE9000E8
:104CD20007F0A3EFF0BE0B04BFB801D3400A900067
:104CE20007740BF0A374B8F0900000E0FAA3E0FBA5
:104CF200EAB52905EBB52A01D3400A900000E5295F
:104D0200F0A3E52AF07F05127C658E2F8F30E4FC3C
:104D1200FD900021E0FEA3E0FF121491C004C00543
:104D2200C006C00774CDFC14FDFE743DFF12112CA9
:104D32008C318D328E338F34E4FCFDAE2FAF3012C6
:104D42001491C004C005C006C007AC31AD32AE3309
:104D5200AF34121288C004C005C006C0077466FED4
:104D6200FCFD743FFF121522BF01028003024E3583
:104D720090000BE0600F14600C1460431460401448
:054D82006078024E3BC9
:104D8700E4FCFDAE2FAF30121491C004C005C0067D
:104D9700C007AC31AD32AE33AF34121288C004C095
:104DA70005C006C0077455FEFCFD743FFF12112CA9
:104DB700121495EF900002F0807AE4FCFDAE2FAF5D
:104DC70030121491C004C005C006C007AC31AD3223
:104DD700AE33AF34121288C004C005C006C00774D2
:104DE700ABFC14FDFE743EFF12112C121495EF90CC
:104DF7000002F0803FE4FCFDAE2FAF30121491C0EB
:104E070004C005C006C007AC31AD32AE33AF3412B3
:104E17001288C004C005C006C007E4FEFCFD743F4D
:0E4E2700FF12112C121495EF900002F080067D
:104E3500E52D900002F01279EDE4FF22E52EB40392
:014E45001359
:104E460090000BE0B404005005E004F08005E49007
:104E5600000BF090000BE0700F7B027A0079F27D78
:104E6600057C41780112081D90000BE0FAB4010F91
:104E76007B027A0079F27D057C41781212081D903A
:104E8600000BE0FAB4020F7B027A0079F27D057C12
:104E960041782312081D90000BE0FAB4030F7B0241
:104EA6007A0079F27D057C41783412081D90000B5A
:104EB600E0B4040F7B027A0079F27D057C417845E7
:104EC60012081D74069000F2F07F027B027A0079C8
:104ED600F212794E024BAB7F017B057A417956126D
:104EE600794EE52EB40110900002E0B52D01D340B5
:0C4EF60006900002E014F0E52EB4020665
:104F02001279EDE4FF22E52EB4030F900002E0B522
:104F120028005006900002E004F0900002E0FBE45A
:104F2200C0E0C0037B027A0079F27D057C4178679C
:104F320012081D1581158174069000F2F07F027B24
:104F4200027A0079F212794E024BAB7F017B057A2D
:104F520041797912794E900000E0FAA3E0BA000399
:104F6200B464005009900000E4F0A37464F090006F
:104F720000E0FAA3E0FBEAB52905EBB52A01D3402C
:104F82000A900000E529F0A3E52AF0E52EB40120FD
:104F9200900000E0B40006A3E0B46401D340119095
:104FA2000001E024CEFB900000E034FFF0A3EBF020
:0A4FB200E52EB40202800302503F16
:104FBC00900000E0FAA3E0FB900007EAF0A3EBF00E
:104FCC00900007E0B40005A3E0B464005009900021
:104FDC0007E4F0A37464F0E4FCFD900007E0FEA38A
:104FEC00E0FF121491C004C005C006C0077C0A7D06
:104FFC00D77E237F3C12112C121495EE900007F0F3
:10500C00A3EFF0900007E0FEA3E0FFE4FC7D641248
:10501C000141EE900007F0A3EFF0BE0B04BFB80106
:10502C00D3400A900007740BF0A374B8F01279ED1A
:10503C00E4FF22E52EB4031F900000E0B52905A380
:10504C00E0B52A005011900001E02432FB900000E2
:10505C00E03400F0A3EBF0900000E0C0E0A3E0C06F
:10506C00E07B027A0079F27D057C41788A12081D7A
:10507C001581158174069000F2F07F027B027A0094
:10508C0079F212794E024BAB7F017B057A40795550
:10509C0012794E900007E0FAA3E0BA0003B4640062
:1050AC005009900007E4F0A37464F0900007E0FA54
:1050BC00A3E0BA0B04B4B801D3400A900007740BF8
:1050CC00F0A374B8F0E52EB40120900007E0B40012
:1050DC0006A3E0B46401D34011900008E0249CFBCB
:0F50EC00900007E034FFF0A3EBF0E52EB40206CE
:1050FB001279EDE4FF22E52EB4031F900007E0B414
:10510B000B05A3E0B4B8005011900008E02464FB39
:10511B00900007E03400F0A3EBF0900007E0C0E054
:10512B00A3E0C0E07B027A0079F27D057C41789A9E
:10513B0012081D1581158174069000F2F07F027B19
:10514B00027A0079F212794E024BAB7F017B057A22
:10515B0040797612794E900009E0FAA3E0BA000389
:10516B00B464005009900009E4F0A37464F0E52ED8
:10517B00B40120900009E0B40006A3E0B46401D3AD
:10518B00401190000AE0249CFB900009E034FFF0F2
:08519B00A3EBF0E52EB40206BF
:1051A3001279EDE4FF22E52EB4031F900009E0B568
:1051B3002B05A3E0B52C00501190000AE02464FBFA
:1051C300900009E03400F0A3EBF0900009E0C0E0A8
:1051D300A3E0C0E07B027A0079F27D057C41789AF6
:1051E30012081D1581158174069000F2F07F027B71
:0B51F300027A0079F212794E024BABF9
:1051FE008F27E4F528752901F52A752B10AE2AAFF5
:10520E002B127A838E2C8F2DE52B2401FFE4352A69
:10521E00FE127A83EF900111F0E52B2402FFE435A4
:10522E002AFE127A83EE900106F0A3EFF0E52B240E
:10523E0003FFE4352AFE127A83EF900108F012077D
:01524E00F46B
:10524F00127A008F2EE52714600E14600B1460087D
:08525F00147003025ADC80E820
:10526700E527B40117C028C0297B027A0179147D8C
:10527700057C4178AA12081D15811581E527B4021E
:1052870017C028C0297B027A0179147D057C4178F3
:10529700BC12081D15811581E527B40317C028C066
:1052A700297B027A0179147D057C4178CE12081D8D
:1052B70015811581E52EB40102800302534AE528C2
:0B52C700B40006E529B40001D34078D4
:1052D200E529152970021528E528B40006E529B448
:0552E2000001D3405D56
:1052E700E52924FFFFE52834FFFEE4FC7D0A1201CF
:1052F70041EF2410F52BE43EF52AAE2AAF2B127AA4
:10530700838E2C8F2DE52B2401FFE4352AFE127A9C
:1053170083EF900111F0E52B2402FFE4352AFE12FA
:105327007A83EE900106F0A3EFF0E52B2403FFE468
:0D533700352AFE127A83EF900108F08006FF
:10534400E4F52875290BE52EB4020280030258BC4B
:10535400E529640B45287003E4FF22E527B4010224
:0553640080030254A5C6
:10536900E5292400FBE5283455F5F0E52CB5F002D4
:0F5379008003025461E52DB503028003025461E5
:105388007F017B057A4179E012794EC028C0297BDC
:10539800027A0179147D057C4178F112081D158186
:1053A80015817F027B027A01791412794EE529244E
:1053B800FFFFE52834FFFEE4FC7D0A120141EF24DB
:1053C80010F52BE43EF52AE52B2401FFE4352AFEEF
:1053D800127A83EF90000BF0E52B2402FFE4352AC4
:1053E800FE127A83EE900000F0A3EFF0E52B240381
:1053F800FFE4352AFE127A83EF900002F0E52B24B1
:1054080004FFE4352AFE127A83EE900007F0A3EF3A
:10541800F0E52B2405FFE4352AFE127A83EE90008E
:1054280009F0A3EFF0E52B2406FFE4352AFE127AF3
:1054380083EE90000CF0A3EFF0127AF3E4FE7F0EF7
:10544800127B46E4FE7F0EAC28AD29127A55127BFA
:09545800691279EDD205E4FF228E
:105461001279ED7F017B057A42790312794EC028CA
:10547100C0297B027A0179147D057C4278141208D7
:105481001D158115817F027B027A01791412794EF3
:10549100E4FE7F641279D51279ED7E057FDC127905
:0E54A100D5E4FF22E527B4020280030257067D
:1054AF00E5292400FBE5283455F5F0E52CB5F0028D
:0F54BF00800302561AE52DB50302800302561A28
:1054CE007B057A427926123ED6EF640160030257BD
:0154DE0006C7
:1054DF007F017B057A42793712794EC028C0297B2C
:1054EF00027A0179147D057C42784812081D1581D6
:1054FF0015817F027B027A01791412794E127AF3A9
:10550F00E52924FFFFE52834FFFEE4FC7D0A1201A4
:10551F0041EF2410F52BE43EF52AAE2AAF2B127B78
:10552F0046E52B2401FFE4352AFE127B46E52B24AA
:10553F0002FFE4352AFE127B46E52B2403FFE435F8
:10554F002AFE127B46E52B2404FFE4352AFE127B4C
:10555F0046E52B2405FFE4352AFE127B46E52B2476
:10556F0006FFE4352AFE127B46AE2AAF2BE529242F
:10557F0000FDE5283455FC127A55E52B2401FFE494
:10558F00352AFE90000BE0FD7C00127A55E52B24A6
:10559F0002FFE4352AFE900000E0FCA3E0FD127A42
:1055AF0055E52B2403FFE4352AFE900002E0FD7C35
:1055BF0000127A55E52B2404FFE4352AFE900007EC
:1055CF00E0FCA3E0FD127A55E52B2405FFE4352A14
:1055DF00FE900009E0FCA3E0FD127A55E52B2406AE
:1055EF00FFE4352AFE90000CE0FCA3E0FD127A5593
:1055FF00E4FE7F0E127B46E4FE7F0EAC28AD29122F
:0B560F007A55127B691279EDE4FF224E
:10561A007F017B057A42793712794EC028C0297BEF
:10562A00027A0179147D057C42784812081D158199
:10563A0015817F027B027A01791412794E127AF36C
:10564A00E52924FFFFE52834FFFEE4FC7D0A120168
:10565A0041EF2410F52BE43EF52AAE2AAF2BE529BB
:10566A002400FDE5283455FC127A55E52B2401FF68
:10567A00E4352AFE90000BE0FD7C00127A55E52BFA
:10568A002402FFE4352AFE900000E0FCA3E0FD12AC
:10569A007A55E52B2403FFE4352AFE900002E0FD4B
:1056AA007C00127A55E52B2404FFE4352AFE90008B
:1056BA0007E0FCA3E0FD127A55E52B2405FFE4354B
:1056CA002AFE900009E0FCA3E0FD127A55E52B249E
:1056DA0006FFE4352AFE90000CE0FCA3E0FD127AF6
:1056EA0055E4FE7F0E127B46E4FE7F0EAC28AD2900
:1056FA00127A55127B691279EDE4FF22E527B40389
:06570A000280030258BCFE
:10571000E5292400FBE5283455F5F0E52CB5F00229
:0F57200080030257FEE52DB5030280030257FEFA
:10572F007B057A42795A123ED6EF64016003025824
:01573F00BCAD
:105740007F017B057A42796B12794EC028C0297B94
:10575000027A0179147D057C4178F112081D1581CA
:1057600015817F027B027A01791412794E127AF345
:10577000E52924FFFFE52834FFFEE4FC7D0A120141
:1057800041EF2410F52BE43EF52AAE2AAF2B127B15
:1057900046E52B2401FFE4352AFE127B46E52B2447
:1057A00002FFE4352AFE127B46E52B2403FFE43595
:1057B0002AFE127B46E52B2404FFE4352AFE127BE9
:1057C00046E52B2405FFE4352AFE127B46E52B2413
:1057D00006FFE4352AFE127B46E52B2407FFE4355D
:1057E0002AFE127B46E4FE7F0E127B46E4FDFEFCA1
:0E57F0007F0E127A55127B691279EDE4FF22CA
:1057FE007F017B057A42796B12794EC028C0297BD6
:10580E00027A0179147D057C4178F112081D15810B
:10581E0015817F027B027A01791412794E127AF386
:10582E00E52924FFFFE52834FFFEE4FC7D0A120182
:10583E0041EF2410F52BE43EF52AAE2AAF2B127B56
:10584E0046E52B2401FFE4352AFE127B46E52B2488
:10585E0002FFE4352AFE127B46E52B2403FFE435D6
:10586E002AFE127B46E52B2404FFE4352AFE127B2A
:10587E0046E52B2405FFE4352AFE127B46E52B2454
:10588E0006FFE4352AFE127B46E52B2407FFE4359E
:10589E002AFE127B46E4FE7F0E127B46E4FDFEFCE2
:1058AE007F0E127A55127B691279EDE4FF22E52EF6
:1058BE00B403028003025950E528B40005E529B46B
:0758CE000C004003025950D9
:1058D5000529E52970020528640C45287006E4F5BC
:1058E50028752901E528B40005E529B40B00505BAE
:1058F500E52924FFFFE52834FFFEE4FC7D0A1201BB
:1059050041EF2410F52BE43EF52AAE2AAF2B127A8F
:10591500838E2C8F2DE52B2401FFE4352AFE127A88
:1059250083EF900111F0E52B2402FFE4352AFE12E6
:105935007A83EE900106F0A3EFF0E52B2403FFE454
:10594500352AFE127A83EF900108F0E529640B45AC
:03595500287015A2
:105958007B027A0179147D057C42787C12081D74DB
:1059680006900114F07F017B027A01791412794EB6
:10597800E52EB404037F0422E5292400FBE528343E
:1059880055F5F0E52CB5F0028003025A9FE52DB5D8
:0759980003028003025A9F85
:10599F00900111E0601514603C14606214700302F2
:0B59AF005A36147003025A5F025A8639
:1059BA00900106E0C0E0A3E0C0E0A3E0FBE4C0E0A1
:1059CA00C0037B027A0179147D057C42788D120826
:1059DA001D74FC2581F581025A86900106E0C0E01B
:1059EA00A3E0C0E0A3E0FBE4C0E0C0037B027A01CD
:1059FA0079147D057C42789F12081D74FC2581F577
:105A0A00818079900106E0C0E0A3E0C0E0A3E0FB5A
:105A1A00E4C0E0C0037B027A0179147D057C4278F8
:105A2A00B112081D74FC2581F5818050900106E0B1
:105A3A00C0E0A3E0C0E0A3E0FBE4C0E0C0037B0257
:105A4A007A0179147D057C4278C412081D74FC25FC
:105A5A0081F5818027900106E0C0E0A3E0C0E0A3C1
:105A6A00E0FBE4C0E0C0037B027A0179147D057C87
:105A7A004278D712081D74FC2581F581900002E056
:095A8A006007900011E0B4011B5B
:0C5A9300742090011AF07441A3F0800F01
:105A9F007B027A0179147D057C4278EA12081D7425
:105AAF0006900114F0E528B40005E529B40B005069
:105ABF000E7F027B027A01791412794E025BE67F28
:105ACF00027B057A4279FB12794E02524F7B057A9F
:0E5ADF0043790C123ED6EF64016003025BE6D1
:105AED007F017B057A43791D12794E7F027B057A02
:105AFD0043792E12794E127AF3127B09E4FE7F64FC
:105B0D001279D5E4FDFEFF7C01127A55E4FE7F018A
:105B1D00900011E0FD7C00127A55E4FE7F029000AA
:105B2D001BE0FD7C00127A55E4FE7F0390001FE020
:105B3D00FD7C00127A55E4FE7F04900020E0FD7C90
:105B4D0000127A55E4FE7F05900018E0FCA3E0FDFD
:105B5D00127A55E4FE7F0690000EE0FCA3E0FD12E4
:105B6D007A55E4FE7F07900021E0FCA3E0FD127A58
:105B7D0055E4FE7F08900015E0FCA3E0FD127A5578
:105B8D00E4FE7F0990001CE0FD7C00127A55E4FED6
:105B9D007F0A90001DE0FD7C00127A55E4FE7F0B1C
:105BAD0090001EE0FD7C00127A55E4FE7F0C900003
:105BBD0012E0FD7C00127A55E4FE7F0D900013E09B
:105BCD00FCA3E0FD127A55E4FDFEFC7F0E127A5522
:0C5BDD00127B691279EDE4FF2202524FA6
:055BE9008F271207F4F4
:105BEE00127A008F28E528B404037F0422E52714D7
:105BFE006014147003025CA5147003025D661470C9
:065C0E0003025DDE80DAF6
:105C14007F017B057A43793F12794E900011E0B4FD
:105C240001117B027A0179287D057C4378501208A2
:105C34001D800F7B027A0179287D057C43786112EF
:105C4400081D7406900128F07F027B027A017928EE
:0E5C540012794EE52864016005E528B40311BD
:105C6200900011E0B40104E4F08006740190001188
:0B5C7200F0E528B402028003025E6A25
:075C7D0090001AE0B4011BC6
:105C8400127AF3E4FE7F01127B46E4FE7F0190006A
:105C940011E0FD7C00127A55127B691279EDE4FF64
:105CA400227F017B057A43797212794EE528B4018B
:015CB40015DA
:105CB50090001BE0B40101D34005E014F0800674A8
:0A5CC5000390001BF0E528B402284C
:075CCF0090001AE0B4011B74
:105CD600127AF3E4FE7F02127B46E4FE7F02900016
:105CE6001BE0FD7C00127A55127B691279EDE4FF08
:065CF60022E528B40314AE
:105CFC0090001BE0B403005005E004F08006740132
:105D0C0090001BF090001BE0B4010F7B027A01792C
:105D1C00287D057C43788312081D90001BE0B4029B
:105D2C000F7B027A0179287D057C43789412081D3B
:105D3C0090001BE0B4030F7B027A0179287D057C6F
:105D4C004378A512081D7406900128F07F027B028F
:105D5C007A01792812794E025BEE7F017B057A433A
:105D6C0079B612794E900010E0FBE4C0E0C0037BE2
:105D7C00027A0179287D057C40782212081D158154
:105D8C0015817406900128F07F027B027A01792834
:105D9C0012794EE528B40110900010E0B40101D343
:0D5DAC004006900010E014F0E528B4020657
:105DB9001279EDE4FF22E528B403028003025E6A4A
:105DC900900010E0B40A004003025E6A900010E0FF
:105DD90004F0025BEE7F017B057A4379C712794EA5
:105DE90090001FE0B401117B027A0179287D057CBE
:105DF9004378D812081D800F7B027A0179287D0526
:105E09007C4378E912081D7406900128F07F027B13
:105E1900027A01792812794EE52864016005E5289E
:035E2900B40311AE
:105E2C0090001FE0B40104E4F08006740190001FA0
:065E3C00F0E528B4022885
:075E420090001AE0B4011BFF
:105E4900127AF3E4FE7F03127B46E4FE7F0390009F
:105E59001FE0FD7C00127A55127B691279EDE4FF8F
:045E690022025BEEC8
:065E6D007524011207F488
:105E7300127A008F25E52514600F14601D146076D7
:095E8300147003025F09025F0CB8
:105E8C00E524B40101D340041524807475240580E5
:065E9C006FE524B40506C9
:065EA2001207F4E4FF22E8
:075EA80090001AE0B401159F
:105EAF00AF241251FE8F26E526B404037F0422305F
:055EBF000536E4FF229E
:105EC4001207F47F017B057A4379FA12794E7F0237
:105ED4007B057A44790B12794E1279EDE4FE7FFA50
:105EE4001279D51279ED7E077FD01279D51207F495
:105EF400E4FF228013E524B405005004052480083F
:105F040075240180037F0422E52414600E14601CB0
:0B5F140014602A1460381460468053AB
:105F1F007B027A01793C7D057C44781C12081D8038
:105F2F00427B027A01793C7D057C44782D12081D55
:105F3F0080317B027A01793C7D057C44783E1208E2
:105F4F001D80207B027A01793C7D057C44784F12BD
:105F5F00081D800F7B027A01793C7D057C447860B7
:105F6F0012081D740690013CF07F017B027A0179C3
:105F7F003C12794E7B027A01793C7D057C44787125
:105F8F0012081D7405900140F004A3F07F027B02FC
:0A5F9F007A01793C12794E025E731C
:065FA9007524011207F44B
:105FAF00127A008F25E525146012146022147003F5
:0C5FBF0002605D14700302606D026070EF
:105FCB00E524B40101D34005152402607075240546
:085FDB00026070E524B4050624
:065FE3001207F4E4FF22A6
:105FE900E52464026005E524B4032990000BE0B4BC
:055FF9000101D3401F6F
:105FFE007F017B057A44798212794E7F027B057A86
:10600E0044799312794E7E077FD01279D5803BE585
:0C601E0024B4032790001BE06401601F05
:10602A007F017B057A44798212794E7F027B057A59
:0F603A004479A412794E7E077FD01279D5800F5A
:10604900AF24125BE98F26E526B404037F042212EC
:1060590007F48013E524B40500500405248008756D
:10606900240180037F0422E5241460181460581465
:10607900700302612E14700302619C1470030261A3
:04608900DE025FAF25
:10608D007B027A0179507D057C4478B512081D7428
:10609D0006900150F07F017B027A01795012794E02
:1060AD00900011E0B4010E7F027B057A4479C6128F
:1060BD00794E0262097F027B057A4479D712794EB7
:1060CD00025FAF7B027A0179507D057C4478E8123E
:1060DD00081D7406900150F07F017B027A01795002
:1060ED0012794E90001BE0B4010B7F027B057A44C0
:1060FD0079F912794E90001BE0B4020B7F027B05FB
:10610D007A45790A12794E90001BE0B403028003A0
:10611D000262097F027B057A45791B12794E025F77
:10612D00AF7B027A0179507D057C45782C12081DD4
:10613D007406900150F07F017B027A01795012793B
:10614D004E90000BE0B40101D3500890001BE064A9
:10615D000160117B027A0179507D057C45783D12F5
:10616D00081D801D900010E0FBE4C0E0C0037B0221
:10617D007A0179507D057C40782212081D15811514
:10618D00817F027B027A01795012794E025FAF7BDB
:10619D00027A0179507D057C45784E12081D7406F2
:1061AD00900150F07F017B027A01795012794E9067
:1061BD00001FE0B4010D7F027B057A45795F1279EE
:1061CD004E80397F027B057A45797012794E025FD8
:1061DD00AF7B027A0179507D057C45788112081DCF
:1061ED007406900150F07F017B027A01795012798B
:0F61FD004E7F027B057A4279FB12794E025FAF2B
:06620C00E4F5211207F485
:10621200127A008F22E52214600C14601C147003A1
:066222000262B10262BF3E
:10622800E521B40001D3400515210262BF752103A1
:106238000262BFE521600B14602714604714606395
:0262480080755F
:0D624A0012480B8F231207F4E523B404580B
:106257001279ED30800320814FE4FE7F641279D5F7
:0F62670080F1125E6D8F231207F4E523B4041249
:106276001279ED308003208109E4FE7F641279D51E
:1062860080F130052422125FA98F231207F4E5233B
:03629600B4041637
:106299001279ED30800320810DE4FE7F641279D5F7
:1062A90080F11207F422800EE521B40300500405A1
:1062B900218003E4F521E521600B1460191460279E
:0562C900146035804265
:1062CE007B027A0179647D057C45789212081D80E7
:1062DE00317B027A0179647D057C4578A312081D15
:1062EE0080207B027A0179647D057C4578B41208A2
:1062FE001D800F7B027A0179647D057C4578C5127D
:10630E00081D7406900164F07F017B027A017964A6
:10631E0012794E7B027A0179647D057C4478711284
:10632E00081D7405900168F004A3F07F027B027AC9
:09633E0001796412794E02621229
:106347007F017B057A4579D612794E7F027B057AE4
:106357004579E712794E7E057FDC1279D57F017B7F
:10636700057A4579F812794E7F027B057A467909D5
:1063770012794E7E057FDC1279D5E4F5211207F4F8
:10638700127A008F22E52214600814601614602622
:02639700803252
:10639900E521B40001D340041521802675210A8026
:0663A90021E521B40A0405
:0463AF001207F422BB
:1063B300AF211268041207F4800EE521B40A0050DD
:1063C3000405218003E4F521E521B40B0040030219
:1063D3006801FA232A9063DC730263FF02644A02B2
:1063E30064950264E002652B026597026603026608
:0C63F3004E0266990267390267D6808866
:1063FF007B027A0179787D057C46781A12081D7424
:10640F0006900178F07F017B027A01797812794E3C
:10641F00900013E0C0E0A3E0C0E07B027A0179783E
:10642F007D057C46782B12081D158115817F027B17
:10643F00027A01797812794E0263877B027A0179A9
:10644F00787D057C46783B12081D7406900178F024
:10645F007F017B027A01797812794E90000EE0C0AD
:10646F00E0A3E0C0E07B027A0179787D057C467875
:10647F002B12081D158115817F027B027A01797815
:10648F0012794E0263877B027A0179787D057C460B
:10649F00784C12081D7406900178F07F017B027A08
:1064AF0001797812794E90001EE0FBE4C0E0C00342
:1064BF007B027A0179787D057C46785D12081D157F
:1064CF008115817F027B027A01797812794E0263FE
:1064DF00877B027A0179787D057C46786E12081DDC
:1064EF007406900178F07F017B027A017978127936
:1064FF004E900012E0FBE4C0E0C0037B027A01790A
:10650F00787D057C46785D12081D158115817F0207
:10651F007B027A01797812794E0263877B027A01C6
:10652F0079787D057C46787F12081D740690017876
:10653F00F07F017B027A01797812794EE4FCFD90AD
:10654F000018E0FEA3E0FF121491C004C005C006BE
:10655F00C0077C6F7D127E837F3A12112CC004C05E
:10656F0005C006C0077B027A0179787D057C4678E5
:10657F009012081D74FC2581F5817F027B027A0140
:10658F00797812794E0263877B027A0179787D05DB
:10659F007C4678A212081D7406900178F07F017B6B
:1065AF00027A01797812794EE4FCFD900015E0FE35
:1065BF00A3E0FF121491C004C005C006C0077C6F92
:1065CF007D127E837F3A12112CC004C005C006C015
:1065DF00077B027A0179787D057C46789012081D39
:1065EF0074FC2581F5817F027B027A01797812791B
:1065FF004E0263877B027A0179787D057C4678B3FA
:10660F0012081D7406900178F07F017B027A0179E0
:10661F007812794E90001CE0FBE4C0E0C0037B02CF
:02662F007A01EE
:1066310079787D057C4678C412081D158115817F06
:10664100027B027A01797812794E0263877B027AA2
:106651000179787D057C4678D712081D7406900172
:1066610078F07F017B027A01797812794E90001DD2
:10667100E0FBE4C0E0C0037B027A0179787D057C10
:106681004678C412081D158115817F027B027A01AB
:10669100797812794E0263877B027A0179787D05D8
:1066A1007C4678E812081D7406900178F07F017B22
:1066B100027A01797812794E900021E0FEA3E0FF81
:1066C100E4FCFD121491C004C005C006C00774CDDE
:1066D100FC14FDFE743DFF12112C8C238D248E259C
:1066E1008F26900020E0FF127C65E4FCFD121491DE
:1066F100C004C005C006C007AC23AD24AE25AF263B
:10670100121288C004C005C006C007900020E0FB3B
:10671100E4C0E0C0037B027A0179787D057C46788C
:10672100F912081D74FA2581F5817F027B027A0135
:10673100797812794E0263877B027A0179787D0537
:106741007C47780C12081D7406900178F07F017B5C
:10675100027A01797812794E900021E0FEA3E0FFE0
:10676100E4FCFD121491C004C005C006C00774CD3D
:10677100FC14FDFE743DFF12112C8C238D248E25FB
:106781008F267F05127C65E4FCFD121491C004C0C4
:1067910005C006C007AC23AD24AE25AF2612128872
:1067A100C004C005C006C007900021E0C0E0A3E01E
:1067B100C0E07B027A0179787D057C47781D12085B
:1067C1001D74FA2581F5817F027B027A01797812A5
:1067D100794E0263877B027A0179787D057C47785F
:1067E1002D12081D7406900178F07F017B027A0159
:1067F100797812794E7F027B057A4279FB12794EC4
:03680100026387A8
:056804008F271207F4CC
:10680900127A008F28E527B40A004003026FB4FA10
:10681900232A90681F7302683F0268F80269B1026F
:106829006A4C026AF6026BD0026CAA026D42026DD2
:06683900DA026EC080CA05
:10683F007F017B057A47793E12794E900013E0C0B5
:10684F00E0A3E0C0E07B027A01798C7D057C46787D
:10685F002B12081D15811581740690018CF07F0293
:10686F007B027A01798C12794EE528B401209000D1
:10687F0013E0B40306A3E0B4E801D3401190001471
:10688F00E024FBFB900013E034FFF0A3EBF0E528CE
:03689F00B4022719
:0768A20090001AE0B4011C94
:1068A900127AF3E4FE7F0D127B46E4FE7F0D900021
:1068B90013E0FCA3E0FD127A55127B691279ED22EF
:1068C900E528B403028003026FB4900013E0B40713
:1068D90005A3E0B4D0004003026FB4900014E02493
:1068E90005FB900013E03400F0A3EBF00268097F88
:1068F900017B057A47794F12794E90000EE0C0E08E
:10690900A3E0C0E07B027A01798C7D057C46782B77
:1069190012081D15811581740690018CF07F027B88
:10692900027A01798C12794EE528B4012090000E83
:10693900E0B40306A3E0B4E801D3401190000FE0EE
:1069490024FBFB90000EE034FFF0A3EBF0E528B444
:02695900022713
:07695B0090001AE0B4011CDA
:10696200127AF3E4FE7F06127B46E4FE7F06900075
:106972000EE0FCA3E0FD127A55127B691279ED223A
:10698200E528B403028003026FB490000EE0B4075E
:1069920005A3E0B4D0004003026FB490000FE024DE
:1069A20005FB90000EE03400F0A3EBF00268097FD3
:1069B200017B057A47796012794E90001EE0FBE474
:1069C200C0E0C0037B027A01798C7D057C46785D4C
:1069D20012081D15811581740690018CF07F027BCF
:1069E200027A01798C12794EE528B4011090001ECA
:1069F200E0B41E01D3400690001EE014F0E528B476
:026A020002266A
:076A040090001AE0B4011B31
:106A0B00127AF3E4FE7F0B127B46E4FE7F0B9000C1
:106A1B001EE0FD7C00127A55127B691279ED22E59E
:106A2B0028B403028003026FB490001EE0FB7A00CF
:106A3B00B4F0004003026FB490001EE004F0026853
:106A4B00097B027A01798C7D057C47787112081DD0
:106A5B007F017B027A01798C12794E900012E0FB58
:106A6B00E4C0E0C0037B027A01798C7D057C46781B
:106A7B005D12081D15811581740690018CF07F0243
:106A8B007B027A01798C12794EE528B401109000C3
:106A9B0012E0B41E01D34006900012E014F0E5287A
:036AAB00B402260C
:076AAE0090001AE0B4011B87
:106AB500127AF3E4FE7F0C127B46E4FE7F0C900015
:106AC50012E0FD7C00127A55127B691279ED22E500
:106AD50028B403028003026FB4900012E0FB7A0031
:106AE500B4F0004003026FB4900012E004F00268B5
:106AF500097F017B057A47798212794E900018E06B
:106B0500FEA3E0FFE4FCFD121491C004C005C0061D
:106B1500C0077C6F7D127E837F3A12112CC004C0A2
:106B250005C006C0077B027A01798C7D057C477814
:106B35009312081D74FC2581F581740690018CF073
:106B45007F027B027A01798C12794EE528B4012007
:106B5500900018E0B40606A3E0B44001D3401190BC
:106B65000019E024F6FB900018E034FFF0A3EBF0E9
:056B7500E528B4022731
:076B7A0090001AE0B4011CB9
:106B8100127AF3E4FE7F05127B46E4FE7F05900056
:106B910018E0FCA3E0FD127A55127B691279ED220F
:106BA100E528B403028003026FB4900018E0B40733
:106BB10005A3E0B46C004003026FB4900019E02417
:106BC1000AFB900018E03400F0A3EBF00268097FA3
:106BD100017B057A4779A412794E900015E0FEA356
:106BE100E0FFE4FCFD121491C004C005C006C0071B
:106BF1007C6F7D127E837F3A12112CC004C005C0C8
:106C010006C0077B027A01798C7D057C4778931257
:106C1100081D74FC2581F581740690018CF07F02BA
:106C21007B027A01798C12794EE528B4012090001B
:106C310015E0B40106A3E0B4F401D34011900016AD
:106C4100E024F6FB900015E034FFF0A3EBF0E5281B
:036C5100B4022763
:076C540090001AE0B4011CDE
:106C5B00127AF3E4FE7F08127B46E4FE7F08900075
:106C6B0015E0FCA3E0FD127A55127B691279ED2237
:106C7B00E528B403028003026FB4900015E0B4045E
:106C8B0005A3E0B4B0004003026FB4900016E024FB
:106C9B000AFB900015E03400F0A3EBF00268097FCB
:106CAB00017B057A4779B512794E90001CE0FBE425
:106CBB00C0E0C0037B027A01798C7D057C4778C6E6
:106CCB0012081D15811581740690018CF07F027BD3
:106CDB00027A01798C12794EE528B4011090001CD0
:106CEB00E0B40501D3400690001CE014F0E528B495
:026CFB0002266F
:076CFD0090001AE0B4011B36
:106D0400127AF3E4FE7F09127B46E4FE7F099000C9
:106D14001CE0FD7C00127A55127B691279ED22E5A4
:106D240028B403028003026FB490001CE0B419007D
:106D34004003026FB490001CE004F00268097F0174
:106D44007B057A4779D812794E90001DE0FBE4C0A8
:106D5400E0C0037B027A01798C7D057C4778C612FA
:106D6400081D15811581740690018CF07F027B0249
:106D74007A01798C12794EE528B4011090001DE057
:106D8400B40301D3400690001DE014F0E528B402DA
:016D940026D8
:076D950090001AE0B4011B9D
:106D9C00127AF3E4FE7F0A127B46E4FE7F0A90002F
:106DAC001DE0FD7C00127A55127B691279ED22E50B
:106DBC0028B403028003026FB490001DE0B40A00F3
:106DCC004003026FB490001DE004F00268097F01DB
:106DDC007B057A4779E912794E900021E0FEA3E019
:106DEC00FFE4FCFD121491C004C005C006C007747A
:106DFC00CDFC14FDFE743DFF12112C9001A012006D
:106E0C00E3900020E0FF127C65E4FCFD121491C0BD
:106E1C0004C005C006C0079001A0121285C004C0B2
:106E2C0005C006C007900020E0FBE4C0E0C0037B77
:106E3C00027A01798C7D057C4678F912081D74FA6A
:106E4C002581F581740690018CF07F027B027A011A
:106E5C00798C12794EE528B40110900020E0B40032
:0F6E6C0001D34006900020E014F0E528B4022680
:076E7B0090001AE0B4011BB6
:106E8200127AF3E4FE7F04127B46E4FE7F04900054
:106E920020E0FD7C00127A55127B691279ED22E521
:106EA20028B403028003026FB4900020E0B404000F
:106EB2004003026FB4900020E004F00268097F01F1
:106EC2007B057A4779FA12794E900021E0FEA3E021
:106ED200FFE4FCFD121491C004C005C006C0077493
:106EE200CDFC14FDFE743DFF12112C9001A0120086
:106EF200E37F05127C65E4FCFD121491C004C00519
:106F0200C006C0079001A0121285C004C005C006C9
:106F1200C007900021E0C0E0A3E0C0E07B027A015C
:106F2200798C7D057C47781D12081D74FA2581F540
:106F320081740690018CF07F027B027A01798C12B7
:106F4200794EE528B4011E900021E0B40706A3E0C3
:106F5200B4D001D3400F900022E014F0F49000214D
:0A6F62007003E014F0E528B40227E4
:076F6C0090001AE0B4011CC3
:106F7300127AF3E4FE7F07127B46E4FE7F0790005C
:106F830021E0FCA3E0FD127A55127B691279ED2210
:106F9300E528B4031C900021E0B40B05A3E0B4B8CA
:106FA30000500E900022E004F09000217003E004F2
:046FB300F002680977
:106FB7002053746172742043686172676572202080
:106FC70000202020202020202020202020202532C3
:106FD700642000205374617274204469736368618C
:046FE7007267650068
:106FEB008E218F228D238D071276AFEE9001C7F085
:106FFB00A3EFF0900034E0FBE49001C1F0A3EBF0C1
:10700B00E4FDFC9001B9F0900021E0FEA3E0FF123B
:10701B0014919001BB1200E3E4FCFD90000CE0FE28
:10702B00A3E0FF121491C004C005C006C0077C6F1B
:10703B007D127E837F3A12112CC004C005C006C09E
:10704B0007900002E0FF7E00E433E4500114FCFDE6
:10705B0012145412112CC004C005C006C0079001B5
:10706B00BB121129121495EE9001C3F0A3EFF0E5BA
:10707B002324FD70030272FD1470030272FD24FEC3
:06708B0060041460012204
:10709100120003AF231276AFEE9001BFF0A3EFF021
:1070A10070189001BFE070129001C7E0FAA3E0FBF5
:1070B1009001BFEAF0A3EBF080109001BFE0FAA3CA
:1070C100E0FB9001C7EAF0A3EBF0E4FCFDAE21AFD9
:1070D10022121491C004C005C006C0077C0A7DD7E6
:1070E1007EA37F3C12112C121495EE9001C5F0A3E2
:0C70F100EFF0E523B40602800302718278
:0E70FD009001BAE0F5F0900032E065F06077A7
:10710B00E09001BAF07B027A0179A47D057C6F785F
:10711B00B712081D74069001A4F07F017B027A015F
:10712B0079A412794EE5FEFF7E00E4FC7D6412012A
:10713B0041E4FC7DFF120155C006C0077B027A01BA
:10714B0079A47D057C6F78C812081D158115818582
:10715B0021248522257B027A0179A49001BFE0FCD2
:10716B00A3E0FD12770674259001B3F07F027B023A
:10717B007A0179A412794EE5FE9001B8F09001BF27
:10718B00E0FAA3E0FBEAFEEBFF9001C6E0F8E52294
:10719B00C398FD9001C5E0FBE5219BFCF5F0EAB53A
:1071AB00F004EFB50500500CE5FEFB7A00B4F300DC
:1071BB00500205FE9001BFE0FAA3E0FB9001C6E090
:1071CB002522FD9001C5E03521FCF5F0EAB5F0056F
:1071DB00EBB50501D3400AE5FEB40001D34002151F
:1071EB00FE9001BFE0FCA3E0FD9001C6E0FAE522B2
:1071FB00C39AFB9001C5E0F8E52198FAF5F0ECB5E0
:10720B00F004EDB50300401EA3E02522FB9001C561
:10721B00E03521FAF5F0ECB5F005EDB50301D350EF
:10722B00058C068D0722E5FEB40101D3400AE5FE6D
:10723B00FB7A00B4F20040099001BFE0FEA3E0FF2F
:0B724B00229001B8E0B5FE01D3401511
:107256009001B9E004F0B40A01D340099001BFE0FF
:0F726600FEA3E0FF2290000BE0B40101D34049EA
:107275001276EFE4FCFD121491C004C005C006C0EF
:1072850007E4FCFD9001C3E0FEA3E0FF121491C0EA
:1072950004C005C006C0079001BB12009CE4FEFCBB
:1072A500FD743FFF12112C120FCC121522BF0109DC
:1072B5009001BFE0FEA3E0FF22E523B407028003AF
:0372C500027091C3
:1072C8003080032081099001BFE0FEA3E0FF2290F7
:1072D80001C1E0FCA3E0FD900034E0FB7A008AF0F5
:1072E800BC0009F5F0ED6B70030270919001BFE0EE
:0572F800FEA3E0FF22EF
:1072FD00120003AF231276AFEE9001BFF0A3EFF0B3
:10730D0070189001BFE070129001C7E0FAA3E0FB86
:10731D009001BFEAF0A3EBF080109001BFE0FAA35B
:10732D00E0FB9001C7EAF0A3EBF0E4FCFDAE21AF6A
:10733D0022121491C004C005C006C0077C0A7DD777
:10734D007EA37F3C12112C121495EE9001C5F0A373
:0C735D00EFF0E523B4030280030273EE9E
:0E7369009001BAE0F5F0900032E065F0607738
:10737700E09001BAF07B027A0179A47D057C6F78F1
:10738700DA12081D74069001A4F07F017B027A01CE
:1073970079A412794EE5FDFF7E00E4FC7D641201BD
:1073A70041E4FC7DFF120155C006C0077B027A014C
:1073B70079A47D057C6F78C812081D158115818514
:1073C70021248522257B027A0179A49001BFE0FC64
:1073D700A3E0FD12770674259001B3F07F027B02CC
:1073E7007A0179A412794EE5FD9001B8F09001BFBA
:1073F700E0FAA3E0FB9001C6E0F8E522C398FD9010
:1074070001C5E0F8E52198FCF5F0EAB5F004EBB525
:107417000500500CE5FDFB7A00B4F300500205FDB2
:107427009001BFE0FAA3E0FB9001C6E02522FD90A2
:1074370001C5E03521FCF5F0EAB5F005EBB505012E
:10744700D3400AE5FDB40001D3400215FD9001BF0A
:10745700E0FCA3E0FD9001C6E0FAE522C39AFB90A9
:1074670001C5E0F8E52198FAF5F0ECB5F004EDB5C3
:107477000300401EA3E02522FB9001C5E03521FA59
:10748700F5F0ECB5F005EDB50301D350058C068D8D
:107497000722E5FDB40101D3400AE5FDFB7A00B4FC
:1074A700F20040099001BFE0FEA3E0FF229001B87F
:0774B700E0B5FD01D3401513
:1074BE009001B9E004F0B40A01D340099001BFE095
:0F74CE00FEA3E0FF22E523B4040280030272FD57
:1074DD003080032081099001BFE0FEA3E0FF2290E0
:1074ED0001C1E0FCA3E0FD900034E0FB7A008AF0DE
:1074FD00BC0009F5F0ED6B70030272FD9001BFE069
:05750D00FEA3E0FF22D7
:107512008E218F22900034E0FBE49001CFF0A3EBA8
:10752200F01276EFEE9001C9F0A3EFF0E4FCFD90CB
:107532000021E0FEA3E0FF1214919001CB1200E3C0
:107542001200031276EFEE9001D3F0A3EFF0701861
:107552009001D3E070129001C9E0FAA3E0FB900120
:10756200D3EAF0A3EBF080109001D3E0FAA3E0FBA2
:107572009001C9EAF0A3EBF090000BE06403600411
:10758200E0B4021E9001CB12009C7C0A7DD77EA340
:107592007F3B12112C121495EE9001D1F0A3EFF063
:1075A200801C9001CB12009C7C0A7DD77EA37F3C7D
:1075B20012112C121495EE9001D1F0A3EFF090016C
:1075C200D3E0FCA3E0FD9001D2E0FAE522C39AFBEE
:1075D2009001D1E0F8E52198FAF5F0ECB5F004ED70
:1075E200B50300500CE5FEFB7A00B4F3005002052F
:1075F200FE9001D3E0FCA3E0FD9001D2E02522FB46
:107602009001D1E03521FAF5F0ECB5F005EDB503C6
:1076120001D3400AE5FEB40001D3400215FE9001F9
:10762200D3E0FCA3E0FD9001D2E0FAE522C39AFB8D
:107632009001D1E0F8E52198FAF5F0ECB5F004ED0F
:10764200B50300401EA3E02522FB9001D1E03521C5
:10765200FAF5F0ECB5F005EDB50301D350058C0653
:107662008D0722E5FE64016006E5FE64F270099072
:1076720001D3E0FEA3E0FF223080032081099001C4
:10768200D3E0FEA3E0FF229001CFE0FCA3E0FD9057
:107692000034E0FB7A008AF0BC0009F5F0ED6B7073
:0D76A200030275429001D3E0FEA3E0FF2239
:0576AF008F2475250089
:1076B400E52424FD601214601E24FE600514600E8F
:0276C400801E26
:1076C6007F06127C65227F07127C652220970F7F3A
:1076D60006127C65222096067F07127C6522052508
:0976E600E525B464C9E4FEFF22AD
:0376EF00752400FF
:1076F2002097067F05127C65220524E524B464F0F8
:04770200E4FEFF2280
:107706008B268A2789288C298D2AE4FCFDAE29AF91
:107716002A121491C004C005C006C007E4FCFD741B
:10772600C8FE7442FF12112CC004C005C006C00773
:10773600E4FCFDAE24AF25121491121288121495A2
:107746008F2BAD26AC27A828AB26AA27A928E4129A
:04775600002A7F0185
:10775A0008E870010CEDFBECFAE8F9740112002A52
:10776A000FBF09EC08E870010CEDFBECFAE8F974BC
:07777A000212002A752C0029
:10778100AF2C7E00E4FC7D0A1201418EF0B2F77449
:0C77910080B5F006E52BB50701D34041A0
:10779D00AB26AA27A928740312002A0528E528700C
:1077AD00020527E52CB40800500CAB26AA27A92802
:1077BD00E412002A800BAB26AA27A9287403120015
:1077CD002AE52CB4090BAB26AA27A9287420120090
:0977DD002A052CE52CB40A9C22BB
:1077E60075FA0075EA0075DA0075FB0075EB007531
:1077F600DB0075FC0075EC0075DC0075FD0075EDB1
:107806000075DD0075FE0075EE0075DE00C2DED285
:0A78160093D294D295D296D2972215
:0B782000EEB40005EFB40001D34007F8
:08782B00EF1F70F11E80EE2238
:10783300C283E4FE7F641278207F3312789B7F3209
:1078430012789B7F2812789B7F0C12789B7F0612FD
:0F785300789B7F0112789B7E017FF412782022B0
:107862008F0553800FED54F04280D283E4FE7F32C5
:10787200127820C28353800FEDC454F04280D28329
:10788200E4FE7F32127820C2837E017FF4127820D8
:0178920022D3
:087893008F3AD28212786222C2
:08789B008F3AC28212786222CA
:1078A3000E1F111111111F000E1F1111111F1F00A7
:1078B3000E1F11111F1F1F000E1F111F1F1F1F005F
:1078C3000E1F1F1F1F1F1F000002060E06020000CF
:1078D30000080C0E0C080000001F1517111F0000F4
:1078E300001F10101010101F001F00000000001FC9
:1078F300001F01010101011F001F1F1F1F1F1F1F69
:107903000E1F11111F1F1F000002060E06020000AA
:1079130000080C0E0C080000001F1517111F0000B3
:107923008F21752240E52175F040A4F521752300D0
:10793300AF2212789BE52125239078A393FF127839
:0B7943009305220523E523B440E62253
:10794E008F358B368A378938EF14600A14600E141F
:06795E0060121460162205
:107964007F8012789B80137FC012789B800C7FFFEE
:0D79740012789B80057FFF12789B7539000B
:10798100AB36AA37A938120071FF1278930538E592
:0D79910038700205370539E539B410E422DD
:07799E0090001FE0B4011C82
:0379A50075210049
:1079A800C2B5E4FE7F281279D5D2B5E4FE7F3C1239
:0A79B80079D50521E521B406E72288
:0779C20090001FE0B4010B6F
:0C79C900C2B5E4FE7F3C1279D5D2B52295
:0479D500EE4F6013FE
:1079D9007B007A06DBFEDAFC7C06E4FDEF1F70EC27
:0479E9001E80E922F1
:0779ED0090001FE0B4010B44
:0C79F400C2B57E037F201279D5D2B522E7
:107A0000E4F53520800375350120810375350220AA
:107A10008006208103753503E53560031279C23095
:057A200080032081211C
:107A2500E4FE7F321279D5E50AB40F01D3400EE5A5
:047A350035B402065C
:107A3900E4F50A7F0422AF3522050A80D9E4F50A64
:037A4900AF352234
:097A4C00C2A3C2A2D2A1D2A02261
:107A55008C2F8D309001D57403F0A374E8F0D2A378
:107A6500EF2400F532EE3405F531AE31AF32127B3D
:0E7A75007FAE2FAF30127BC4127C07C2A3225B
:107A83009001D57401F0A3742CF0D2A3EF2400F578
:107A930030EE3406F52FAE2FAF30127B7F127AAE65
:0B7AA3008E318F32C2A3AE31AF322211
:0F7AAE00E4F533F534F53575360FE53520E7315E
:107ABD00127C31A2A0E4335401753700F538AB3890
:107ACD00AA37A836088005C333CA33CAD8F9453456
:107ADD00F534EA4533F533E536153670CE15358078
:067AED00CAAE33AF3422E3
:107AF3009001D57403F0A374E8F0D2A37E047FC091
:067B0300127B7FC2A322E9
:107B09009001D57403F0A374E8F0D2A37E047F80BA
:097B1900127B7F127C07C2A3223B
:107B22008E088F099001D57403F0A374E8F0D2A3F4
:107B32007E047F40127B7FAE08AF09127BC4127CA9
:047B420007C2A322B1
:107B46009001D57403F0A374E8F0D2A3EF2400F5F6
:107B560030EE3407F52FAE2FAF30127B7F127C0745
:037B6600C2A32295
:107B69009001D57403F0A374E8F0D2A37E04E4FF76
:067B7900127B7FC2A32273
:0F7B7F008E338F34E4F53575360AE53520E7335C
:107B8E00AB34AA33E533A836088005C313CB13CB29
:107B9E00D8F9EB5401753700F53864014537700498
:107BAE00D2A18002C2A1127C31E536153670CC15F9
:067BBE003580C8C2A122BF
:0F7BC4008E338F34E4F53575360FE53520E73312
:107BD300AB34AA33E533A836088005C313CB13CBE4
:107BE300D8F9EB5401753700F53864014537700453
:107BF300D2A18002C2A1127C31E536153670CC15B4
:047C03003580C822DE
:107C0700C2A39001D5E0FEA3E0FF127C4CD2A3747F
:107C1700FFFAFB20A013EA6480B48004BB0001D301
:0A7C27004007EB1B70ED1A80EA2203
:107C3100D2A29001D5E0FEA3E0FF127C4CC2A2903B
:0B7C410001D5E0FEA3E0FF127C4C2206
:107C4C00E4FAFB8EF0EAB5F0068FF0EBB5F00050DD
:097C5C00070BEB70EE0A80EB222D
:107C65008F359001D81200EF00000000E49001D795
:017C7500F01E
:107C7600E4FE7FC8127820AF35127CC9EE9001DC95
:107C8600F0A3EFF09001D812009CE4FCFD9001DC1B
:107C9600E0FEA3E0FF12012C9001D81200E3900150
:107CA600D7E004F0648070C875F007A31200D712FD
:107CB60001179001DCEEF0A3EFF09001DCE0FEA3EB
:037CC600E0FF22BA
:107CC900EF441823232354F8FFD2A40000D2A700BD
:077CD90000C2A700007E05B8
:107CE000C2A4EF30E704D2A68002C2A6EFC333FFDE
:107CF0000000D2A40000DEE8D2A6C2A40000D2A4F4
:0A7D00000000C2A40000E4FF7E05AD
:107D0A00EFC333FF30A5034401FFD2A40000C2A48D
:0D7D1A000000DEECEF540FFCE4FFFD7E08DE
:107D2700EFC333FF30A5034401FFD2A40000C2A470
:0D7D37000000DEECEF2DFFE43CFED2A722A1
:00000001FF
